:020000040800F2
:10500000D81A0020D5500008498C000821830008D8
:105010000000000000000000000000000000000090
:10502000000000000000000000000000DD98000803
:105030000000000000000000D9910008F599000868
:10504000E7500008E7500008E7500008E750000864
:10505000E7500008615D0008E7500008E7500008CD
:1050600000000000E7500008895C0008E7500008D5
:10507000E75000083988000800000000E7500008E9
:1050800000000000E75000080000000000000000E1
:10509000E750000800000000E7500008E750000853
:1050A000E7500008E7500008E750000881A4000816
:1050B000E7500008E7500008000000000000000072
:1050C0000348854600F02CFD0048004701B8000861
:1050D000D81A00200448804704480047FEE7FEE74E
:1050E000FEE7FEE7FEE7FEE7919A0008C1500008E0
:1050F00030B50B46014600202022012409E00D4670
:10510000D5409D4205D31D469540491B25469540F7
:1051100040191546521E002DF1DC30BDF0B51FB40C
:105120000646002082B005464024019100901BE015
:10513000019922460F46304600F0DCFB049A059B9D
:10514000801A994110D310461946224600F0C2FB3E
:10515000361A8F410197224601200021009F00F05E
:10516000B9FB38184D4100902046641E0028DFDC52
:10517000019B00982946324607B0F0BD03460B4319
:105180009B0703D009E008C9121F08C0042AFAD2FD
:1051900003E00B780370401C491C521EF9D2704783
:1051A000D2B201E00270401C491EFBD270470022BF
:1051B000F6E710B513460A4604461946FFF7F0FF16
:1051C000204610BD30B504460020034600E05B1CBD
:1051D000934203D2E05CCD5C401BF8D030BDF8B503
:1051E00002464A40D40F42004B0052085B089A42E4
:1051F00002D20246084611464A0023D0C30D4A0097
:10520000DDB2120EAD1A202D35DA49020126490A07
:10521000F6058A19002C00D0524220214F1B11465E
:10522000B9402A411018C20D9A4221D0002C17D043
:10523000012D08DCDA05801AD20F8019D207DBB203
:1052400000F084FBF8BDDA05801A012340001B063C
:10525000C01880185A428018CA0F1043490007E04E
:105260004908C2071143DA05801A801940088018DE
:1052700000F064FBF8BD61000122511A001BF7E742
:105280000122D2075140AAE70122D2075040A6E7E7
:10529000024670B54A40D30FDB0740002DD04A00CC
:1052A0002AD0010E140E000212020919400A520AF5
:1052B0008418E50104465443000A120A2E045043A0
:1052C000A4194219200CC543AA18120C0125AD03DC
:1052D000521C521912047F39240400D0521C10436E
:1052E00001D44000491EC2B20C06C0092018401C5F
:1052F0004008802A02D003E0002070BD4008400032
:10530000002900DA0020184370BD70B502464A40FB
:10531000D50F40004A00ED0740085208002814D07D
:10532000002A12D0C40DD30D41020120C005520243
:10533000490A520AE41A091812187D34914201D31D
:10534000641C00E04900002C01DA002070BD00233D
:10535000914201D3891A0343400849000028F7D13C
:1053600000290AD0914202D10121C90705E09142EA
:1053700001D2012101E00121C943E005C018401913
:1053800000F0DCFA70BD420005D04200120E52421D
:105390008A4201DB00207047C905081870470000E9
:1053A000F0B507460846584087B0C00F0490480043
:1053B0000E46590040084908BC1A884105D23846B3
:1053C00031461E4617460B46024658004008104319
:1053D0004CD0300D039040055900400D490D05900B
:1053E000401A0290402872DA18030121000B0905C7
:1053F0000843019004980092002805D00199524278
:105400000020884100920190029840210A1A0199D7
:10541000009800F05FFA05460C466B4607CB00F09B
:105420007AFAC0197141039A0E0D0023D71756401E
:105430001A467A40164344D0049A002A2DD0029A84
:10544000012A039A15DC1205C01A9141012636057E
:10545000001C7141D20F059ED20700930192029663
:105460002A46234600F0B8FA07B0F0BD3846314668
:10547000FAE71605224A0F46B218C01AB7410121B1
:105480000905001C4F4100187F4111461818794149
:10549000E20F10436D19644113E0E2076D081543F4
:1054A0006408C2071443039A01261205C01A9141E9
:1054B0003605001C7141CE07400830434908C0182A
:1054C00051412A46234600F07AFACDE7FFE70498D7
:1054D00001224000C117121A00238B410498314663
:1054E000C417381AA141EEE730B40124E407634041
:1054F00030BC55E730B40124E407614030BC4FE7CD
:105500000000E0FFF0B51FB488B00B9909980024A3
:1055100048400999C00F490049080991C0070B99F3
:105520000090490049080B9109990898A64608433C
:105530001CD00B990A98084318D009980124400000
:10554000420D4800410D099824050003000B20433B
:1055500009900B980003000B20430B9050181C4936
:105560004018002201901446104605E00020014634
:105570000DB0F0BD032801DA034600E003239C468A
:10558000C11A0AAE0AE05F0008ADED5B4F00F75BA1
:105590007D430027AA187C41491C5B1E6145F2DD52
:1055A000410004AB5A522104120C0A43240C401C43
:1055B0000828DFDB01980290009970460191009065
:1055C000059B049A0799069800F006FAD0E70000B8
:1055D0000DFCFFFFF0B50C465C4085B0E40FE4071E
:1055E00003944C000026640859009446490802467A
:1055F0000296224321D062460A431ED06200570D14
:105600004A000E032303550D012402462C492405AC
:10561000781B1B0B360B4018234326436146009032
:105620001C46501AB44103D30098401C009002E07D
:10563000921800985B41002803DA0020014605B06B
:10564000F0BD0020012109050746864611E06446A9
:105650001D46141BB54106D36546521BB341744623
:1056600007430C43A646CD07400849082843921833
:105670005B4105460D43EAD11046184313D06046FE
:10568000194650407140084306D06046101AB34195
:1056900006D20122002306E000220123DB0702E0FC
:1056A0000122D2435310009874460105381C614111
:1056B000029C039D0019694100F081F9BFE70000D9
:1056C000FD03000070B54B005B0803430BD04B009B
:1056D0005C0D002633466542B341D417AD1AA34191
:1056E00002DB0020014670BD12053018514170BD2B
:1056F000C217C10F504010B54018CA0796230021A9
:1057000000F024F910BD10B500229623114600F0D8
:105710001DF910BD0EB5C217C10F5040CA07401881
:105720000021054B0293019200910A460B4600F0BE
:1057300053F903B000BD0000330400000EB5054965
:105740000291002100910A460B46019100F044F9B4
:1057500003B000BD33040000C20F4100400201232A
:10576000400ADB05D207090EC0187F2901DA0020A4
:105770007047962903DC9623591AC84001E09639F0
:105780008840002AF4D04042704741004002012284
:10579000400AD205090E80187F2901DA00207047DF
:1057A000962903DC9622511AC840704796398840E2
:1057B0007047000070B5CD0F4A0009030123090BA3
:1057C0001B0519430B4BED070024520D9A4201DAD9
:1057D000002070BD074B34339A4203DC9A1A00F064
:1057E00089F802E00449511888402C43F1D0404226
:1057F00070BD0000FF030000CDFBFFFF4A0009035E
:105800000123090B1B051943094B10B5520D9A4290
:1058100001DA002010BD064B34339A4203DC9A1A99
:1058200000F068F810BD03495118884010BD000011
:10583000FF030000CDFBFFFFC20FD207400040086E
:105840000BD0C10D0723DB01C91840020905400A2E
:105850001143C208400711437047002001467047BA
:1058600010B5002904DB0124E40740428C412146A5
:10587000002B04DB1C460123DB075242A341994263
:1058800000D1904210BD0000CB0FDB07490010B5DE
:10589000490802460A4307D00A0D07240903E40118
:1058A000090B121B002A01DC002010BDC900440FA7
:1058B0000C43C100E018D205801800F03FF810BD7D
:1058C0000122D207002800DB101A002900DB511A40
:1058D0008142704710B5202A04DB0146203A9140EE
:1058E000002010BD914020239C1A0346E340194339
:1058F000904010BD10B5202A04DB0846203AD04065
:10590000002110BD0B46D340D0402024A21A914064
:105910000843194610BD10B5202A06DBCB170846F0
:10592000203A1041C1170B4306E00B461341D0400B
:105930002024A21A91400843194610BD002904DA18
:10594000401C490001D140084000704770B4002459
:10595000050C05D11024000402D1002921D0112406
:10596000050E01D100020834050F01D10001241DEC
:10597000850F01D18000A41C002801DB4000641CBD
:10598000002908D020252E1B0D46F540A14000D04F
:1059900001212943084301061B1B000ADB1D02D518
:1059A000002070BC7047DB05181880180029F8DA51
:1059B000401C4900F5D170BC40084000704710B54C
:1059C000002B08DA0024401C614192185B411A4305
:1059D00001D14008400010BDF0B51FB482B00546AB
:1059E0000C0003D0084604F005FE02E004F002FEBD
:1059F00020300246009021462846FFF76BFF049BAB
:105A0000059A04460F4618431143084314D018461C
:105A100010431BD0009840210A1A18460599FFF739
:105A200069FF05460E46009A05990498FFF752FF54
:105A3000084305D0012004E02046394607B0F0BDF8
:105A40000020C11705430E432C43374300990E989D
:105A50006305401A7905E40A00220C43FD0A0A3066
:105A600002D500200146E9E70105101969410C9CA7
:105A70000D9D00196941FFF7A2FFDFE7FEB5002386
:105A80001A461B1A8A4103DB0020014603B0F0BD11
:105A90004A000D0301212D0B0905520D0D43D107BD
:105AA00002D100186D41521E5110FF31FF310131FA
:105AB000002704463E4638460097019102460121E0
:105AC00000200905FFF716FFC3197141F818324687
:105AD00084468E464A4161462846611A904104D365
:105AE0006046241A954176461F46241900986D4158
:105AF000401C00903428E1DDF91930467041091B43
:105B0000A84103D20022D243134601E000221346EB
:105B100001980105381C7141FFF751FFB6E70000FD
:105B2000064C0125064E05E0E36807CC2B430C3CF0
:105B300098471034B442F7D3FFF7C6FAF0C600080E
:105B400010C7000870B58C180578401C6B075B0FF8
:105B500001D10378401C2A1106D10278401C03E0D1
:105B600006780E70401C491C5B1EF9D12B0705D42A
:105B70000023521E0DD40B70491CFAE70378401C19
:105B8000CB1A921C03E01D780D70491C5B1C521E41
:105B9000F9D5A142D8D3002070BD000038B5044625
:105BA000064805490068FFF7A3FA604300E0401E7D
:105BB00000900028FBD138BD40420F004801002072
:105BC000F8B50446006881688907890F012902D168
:105BD0000168C90722D18168114A102611400125A8
:105BE00000290ED18168294381600120FFF7D6FF8B
:105BF00000F0FAFF07460CE000F0F6FFC01B0A2891
:105C000007D9606D30436065A06D2843A065012011
:105C1000F8BD20680068C043C007EDD10020F8BD82
:105C2000170000801FB50B4800900B4801900B48EF
:105C300002900B48039069460A4805F0D1F80A4AD9
:105C400008481146083904F0B9FF00F04BFA00206B
:105C500004B010BDFDC40008D9C4000839C500084F
:105C600037C50008540100201000002010B50023A3
:105C70001A4603E0845CE3189BB2521C8A42F9D3B3
:105C8000D84380B210BD000010B5034800F068FD95
:105C9000024800F065FD10BD781600203016002087
:105CA00030B5446C1C252C400125A540046C656072
:105CB000046863608368102B036803D099600068F0
:105CC000C26030BD9A600068C16030BD14490120D7
:105CD00048720A4602205E32507203203C3A5072EB
:105CE00004200E3A50720F480D4B00780870223194
:105CF0000870203108770C495A1C08785871497887
:105D000099712333187159712033187759771075A9
:105D100051751A461E3210755175107651767047BE
:105D2000AC110020F70000201801002010B503F08E
:105D3000ABFD202003F054FE012005F0BBFA00204B
:105D400003F04EFE044805F059F9044805F008FC3C
:105D5000002005F03DFC10BDE00000208380000025
:105D6000F8B505200121000700F02AFF0025174C97
:105D7000002800D06560164E0221304600F020FF5A
:105D800000281BD1012020701248808F00280ED0DF
:105D90000127BF0200223946304600F01EFF0A20CC
:105DA00004F07CFE01223946304600F016FF0A4816
:105DB000656000880A21484308490880012000F0F6
:105DC00037FE022000F034FEF8BD00003401002050
:105DD00000040050AC0D002004010020160100203A
:105DE0007047000010B5084900224A6107494B6816
:105DF0004C1523434B604B68082423434B60C00978
:105E0000C001026010BD0000C0160020002002404A
:105E10007FB500250C460646039500F0D9FDE00944
:105E2000029003A901960095684600F069FD0028DC
:105E300004D000F0A1FD002004B070BD00F09CFD76
:105E40000120F9E710B5002302E0C45CCC545B1CD0
:105E50009342FAD310BD000010B5214A0021906989
:105E6000C305204804D541690223194341619115B6
:105E700093699B0505D5436901242343436163026C
:105E8000194393695B0505D543690824234343619E
:105E9000E301194393691B0505D543690424234392
:105EA00043616302194393699B0405D54369102438
:105EB000234343616302194393699B0304D54469F7
:105EC00020231C43446119439369DB0305D54369CF
:105ED000402423434361A0020143916110BD0000AF
:105EE00000200240C016002070B5054600F07CFE80
:105EF0000646184C0AE0681C08D0002D04D000F0BB
:105F000073FE801BA84201D9032070BDA069C007A1
:105F1000F1D1A069800701D50220A061A069C00568
:105F200011D4A06980050ED4A06940050BD4A069E6
:105F3000000508D4A069800405D4A069800302D4B8
:105F4000A069C00303D5FFF787FF012070BD0020C3
:105F500070BD000000200240F8B517460026054637
:105F60000C4600F035FD09E029460220226800F0C9
:105F700011FD002804D1241D2D1D361DBE42F3D372
:105F800000F0FAFCBE4201D20020F8BD0120F8BDAD
:105F900010B5084902460020054B497905E0440048
:105FA0001C5B944203D0401CC0B28842F7D310BDA2
:105FB000D41200207000002010B500F006FE10BDC5
:105FC00010B5094801F030F880B2FFF7B7FB074A77
:105FD000074BFFF797FA0022064BFFF7FBFAFFF794
:105FE0000DFC80B210BD0000E4140020F853E3A5BE
:105FF0009B843E4000408F4070B5364C3448A083AF
:106000003548217F0175617F417534490A780276F0
:106010004978417630490520133148720A2005F04D
:106020008FFA7D20C00005F0A5FA2B49002213311C
:106030000C2005F06FFB00210C2005F07DFB0220F9
:1060400005F0CEFA264D00210F2005F0F9F928427F
:106050002063F8D0206B411C38D0400435D5812214
:10606000D20100210F2005F02AFB0021102005F0AD
:10607000E7F941061848490E0022633005F016FA88
:10608000154D6335687A05281FD102221349681D12
:10609000FFF798F8002818D10E48AE7C66710422EC
:1060A000691C4830FFF76AF8294613310846720028
:1060B0000D465130FFF762F86079294642000648E4
:1060C000DF30FFF75BF80320207070BD04F006FBA3
:1060D00024970000700000200D12002018010020FD
:1060E00000D027240F4A10B5114608390E4804F095
:1060F00065FD0C4C0022103C0C4BE168A068FFF7DA
:1061000069FA0B4A0B4B05F089FC00220A4BFFF79A
:10611000F1F90022094BFFF7F5F9FFF7B5FB206015
:1061200010BD0000100000205401002000AA8F4084
:106130006C45D9CC955BC83F0000F03F40A5E540D9
:1061400010B5084800F096FA0A21064800F032FA25
:10615000044800F01DF9800503D5024800F01AF943
:1061600080B210BD88140020F8B52F4D0022012107
:10617000284600F032FDFFF7E3FFFFF7C4FA2B4E8D
:106180003146FFF7C2F82A4C0122A060114628468A
:1061900000F023FD2749A068002588423EDB2078D7
:1061A000254F002815D02570FFF7CAFFFFF7ABFA7F
:1061B0003146FFF7AAF8A060FFF73EFB00223B46FE
:1061C000FFF792F900221D4BFFF79CF9FFF75CFBEC
:1061D0006060A068FFF730FB00223B46FFF784F9C0
:1061E000174A184BFFF78EF906460F466068FFF70F
:1061F00023FB134A144B5242FFF784F932463B46C5
:10620000FFF7CEF8FFF740FB10496060884201DDE0
:10621000616004E0FF21C905C84200D36560606881
:10622000FFF7B3FAC0B2F8BD0004005000401B44B1
:10623000480000200000604000000C4000E0644086
:106240003333333333B33040CCCCEC3F0000C8425F
:10625000F8B5054604464035287C0026012808D0BC
:1062600001202874206881688907890F01290ED1CF
:1062700001E00220F8BD0168C90708D0606D202147
:10628000084360650126002028743046F8BD616D22
:10629000FF2201329143022211436165C1688907DF
:1062A000890F0091C16889088900C16020688168F0
:1062B00092071143816000F097FC07460EE000F062
:1062C00093FCC01B0A2809D9606D02218843102164
:1062D00008436065002028740120F8BD20688068AC
:1062E0000028ECDB2068C168009A1143C160606D32
:1062F00080088000401C6065C5E70000F8B50646D0
:106300000D464036317C01290DD0012131740168E0
:106310008A68520709D5416D20221143416500204A
:1063200030740120F8BD0220F8BD174B6A68D8050B
:1063300047109A42154C8A6A2B6812D05B035B0B9C
:106340001A438A622968490305D5A1680143A160FF
:106350000A20FFF723FC2868800312D5A068384381
:106360000EE05B035B0B9A438A622968490302D5FE
:10637000A1688143A1602868800302D5A068B84362
:10638000A06000203074F8BD01100000002701401B
:10639000406D70470068006C7047000070B50400E5
:1063A00006D0606D264600254036002802D006E063
:1063B000012070BDA5653574204600F0D3F8606DEE
:1063C000C00603D421688868400705D5606D102198
:1063D000084360653574EBE7606DFF22013290433E
:1063E00002221043606588688207920F5B48012A89
:1063F00002D10A68D2072BD1032362689B079A4215
:1064000005D05B429A4202D05B009A4209D10A69E8
:10641000920092080A6121680A6963681A430A6156
:106420000CE00A69920092080A6181680F229204C6
:106430009143816081686268114381602168CA6804
:1064400018239A43CA602168CA68A3681A43CA60BD
:10645000816801225206914381608168A28E5206B2
:106460001143816020688168C90004D481680122D9
:106470001207114381602068C168394A1140C16028
:106480002069E168022825D0002001432046203001
:106490000278037B52035B001A431143226B1143C2
:1064A000A26992031143E269D20311432268D368BF
:1064B0001943D160616A0A46FF3AC23A05D0A26A1E
:1064C00011432268D3681943D16042780121012A1F
:1064D00002D00BE00420D8E70078002823D0606DBC
:1064E000202210436065A06D0843A065E06B012881
:1064F00020681FD00169C90703D001694908490014
:10650000016120684169C908C90041612068416989
:10651000A26B11434161A565606D80088000401C3D
:106520006065002070BD2068C26801231B041A4307
:10653000C260DBE70269FF239B009A430261206887
:106540000269236CA66C1A43636C33431A430261DD
:10655000206802690A430261D3E700000027014076
:106560001902FEFF10B586B0044614216846FEF7F6
:106570001EFE0E492068884216D10D48416B421517
:1065800011434163C16A01221143C162C06A694675
:1065900010400590022000900320019000200290FE
:1065A0000520000700F050FA06B010BD002401409D
:1065B00000100240F8B504464069254640350E46B5
:1065C00008280BD02068C068C00709D0606D202162
:1065D00008436065002028740120F8BD082700E00A
:1065E0000C2700F001FB009011E0701C0FD0002E72
:1065F00005D000F0F9FA0099401AB04207D9606D51
:10660000042108436065002028740320F8BD206839
:1066100000683842E9D0606D012149020843606595
:106620002068C16809058A0F0C21002A1BD120228D
:10663000125D002A17D10268120714D58268530729
:106640000122002B08DB43688B434360606D13021B
:1066500098431043606506E0606D20231843606531
:10666000A06D1043A065A069002801D120680160D9
:106670000020F8BD70B504462168002089684907EC
:1066800021D425464035297C01291CD001212974BB
:10669000E169012904D02046FFF792FA002811D1C0
:1066A000616D0A4A1140FF220132114361650021E8
:1066B000A165297422681C21116021688A6804235D
:1066C0001A438A6070BD022070BD0000FEF1FFFF1A
:1066D00030B5014620314A790023022A04D0042231
:1066E000C2630B71012030BD026814680E25AC43F3
:1066F000146002681468640864001460446C1C220E
:10670000144001221546006CA54045604A711846A8
:106710000B7130BD70B50024014620314A79022A40
:1067200003D00421C163012418E0026813680E2518
:10673000AB431360026813685B085B001360436C33
:106740001C221340012215469D40036C5D604A7176
:1067500000220A71816B002900D08847204670BD55
:10676000F0B4016C0D6801680C68466C1C230422AF
:106770001E401746B7402F420ED067070CD50C6855
:10678000A40602D40C6894430C60416C19408A4002
:10679000016C4A60016B1AE00227B74002462F40A5
:1067A0002032002F17D0A70715D50C68A40605D4F2
:1067B0000C680A25AC430C6001215171446C022124
:1067C0001C40036CA140596000211171C16A00296D
:1067D00018D0F0BC08470827B7402F4212D0240732
:1067E00010D50C680E25AC430C60446C01211C4094
:1067F0000B46A340046C6360C163517100211171A9
:10680000416BE4E7F0BC704770B504003CD01F4812
:10681000256814212818FEF76BFC800060641C4872
:10682000206402212046203002464171296819481F
:10683000E3680140A068666918432369334318433D
:10684000A3691843E3691843236A1843084328607F
:106850000121A0688903884210D00D488030836AE6
:10686000656C1C210D400F26AE40B3438362656CFE
:1068700063680D40816AAB400B4383620020E06394
:1068800001215171107170BD012070BDF8FFFDBF75
:10689000000002400F80FFFFF8B504468C46203010
:1068A00001790025012909D00126067141790027C7
:1068B000012905D0077102252846F8BD0220F8BD40
:1068C00002214171E76320680168490849000160BD
:1068D00061462046FFF7E4F9206B00282068016834
:1068E00001D00E2205E00422914301602068016876
:1068F0000A22114301602068016831430160DBE72F
:10690000F8B51A4E0546307C0F46012807D0012005
:1069100030741748FFF7E8FA010002D021E00220A6
:10692000F8BD0020C04338606C6814E02046FFF7D3
:1069300059FA0F48FFF7D8FA01460E484268082373
:106940009A434260426843159A434260002901D04D
:106950003C6006E08034A8686A68C0018018A042E4
:10696000E4D8002030740846F8BD0000C0160020AE
:1069700050C3000000200240054841680222114334
:1069800041604168012211434160002070470000CE
:1069900000200240F8B50C4C1646207C0F4601281A
:1069A00008D0012020740948FFF79EFA002500282E
:1069B00002D006E00220F8BD65613E600348FFF7A3
:1069C00093FA2574F8BD0000C016002050C30000E3
:1069D00011484168C9070BD0EFF3108172B60F4A16
:1069E000C2600F4AC26081F310884168C9070ED1A6
:1069F000416889070DD5EFF3108172B6094A02612B
:106A0000094A026181F310884068800701D501209E
:106A1000704700207047000000200240EFCDAB8996
:106A200005040302BFAE9D8C1615141370470000B9
:106A300010B504494A69024202D04861FFF7F6FFE7
:106A400010BD000000040140FCB500230124A2E0B9
:106A500027462A469F403A406FD04D68012D05D009
:106A6000022D03D0112D01D0122D16D185680326D9
:106A7000AC465D00AE46AE406546B543AC46CE681A
:106A80007546AE4065462E43866046680D79BE4326
:106A9000ED06ED0F9D4035434560C6685F00032558
:106AA000BD40AE46AE4335468E68BE402E43C660FE
:106AB0004E68022E01D0122E14D1DE08B600361810
:106AC0000196366A5D07B446EE0E0F25B540009676
:106AD0006646AE43B4460D69009EB54066462E43F9
:106AE000019D2E6206687546AE430D79AD07AD0F68
:106AF000BD40354305604D68ED004BD5294D6E6BAB
:106B000026436E639E08284DB6007519AC46AD68E5
:106B10009E07360F0F27B740BD4305273F07B842F2
:106B200001D1002715E0214FB84201D1012710E023
:106B30001F4FB84202D102270BE02BE01D4FB84295
:106B400001D1032705E01C4FB84201D1052700E021
:106B50000627B7402F436546AF60184D2E684F6833
:106B60009643FF0300D516432E606E684F68964328
:106B7000BF0300D516436E60AE684F689643FF02B0
:106B800000D51643AE60EE684F689643BF0200D54D
:106B90001643EE605B1C0A681546DA4000D057E7E2
:106BA000FCBD000000100240000001400004005045
:106BB00000080050000C0050001C00500004014070
:106BC0000069084000D001207047426913460B401D
:106BD0001B0491430B4383617047002A01D08161FC
:106BE000704781627047000001488068704700006C
:106BF0003C01002002488168027889188160704752
:106C00003C01002010B508480024016840221143CF
:106C10000160204600F00AF8002801D0012401E0BC
:106C200000F04CFA204610BD0020024070B504462A
:106C30000D4D7D202978C000FEF75AFA01460B4819
:106C40000068FEF755FA00F035FF002809D1042C42
:106C500007D200222146401E00F058FA00206C6046
:106C600070BD012070BD00003C01002048010020E3
:106C700070477047F8B5644CA078401CA0700120A4
:106C80002071A08B401CA0836048008802F064FE45
:106C90005F48C088FEF737FD5E49FEF736FB5E4D64
:106CA00006462968FEF79BFA28600120A16AC00504
:106CB000814201DA084603E03046FEF7E5FAA062B9
:106CC000FF21C9050025C84200D3A56260780028CD
:106CD0000BD102215148FFF773FF02005049514880
:106CE00017D00022FFF779FFA56302214B48FFF779
:106CF00067FF002855D0A563454FB88AFEF703FD0E
:106D0000454E3168FEF7DCFD5DD247490120087031
:106D10005BE00122D1034348FFF75FFF3C48C08896
:106D2000FEF7F1FC3B49FEF7F0FAA16BFEF757FACC
:106D30003E49A0638842D8DD35480127F926403016
:106D400000900A213046FEF7D3F9002903D13449D7
:106D50003448FFF731F902213048FFF731FF0028AE
:106D600001D0002701E0002F12D102212B48FFF7AC
:106D700027FF00280CD104F019FE0099012088801B
:106D800005F070FB642003F089FE2A492848C8609A
:106D90000A2003F083FE3046761EF6B20028D0D1DA
:106DA000A3E71B48C088FEF7AEFC1A49FEF7ADFA10
:106DB000A16BFEF714FA2049A06388429CDB1D49B1
:106DC0001B48C86098E718480570788F401EFEF78A
:106DD0008FFC3168FEF774FD06D86079002803D077
:106DE00016490120087001E014480570788FFEF7FD
:106DF0008AFC3168FEF764FD04D26079002801D076
:106E000004F098FDF8BD0000F40000208A00002086
:106E1000AC0D002000007A4438010020000400502E
:106E2000008000000000005076000020000040407C
:106E30000400FA0500ED00E00000A04083000020FF
:106E4000704770B5040010D0022025462035A87385
:106E5000204601F0F9FCA87B032805D0204600F06D
:106E6000B9F80020A873687370BD012070BD704729
:106E7000704710B5044600680168C943C90708D1C6
:106E80008168C943C90704D1012141602046FFF749
:106E9000F1FE20680168C943890708D48168C943A5
:106EA000890704D4022141602046FFF7E1FE2068F3
:106EB0000168C943490708D48168C943490704D414
:106EC00004214160204600F0F7F820680168C943BA
:106ED000090708D48168C943090704D4082141601F
:106EE0002046FFF7ADFF20680168C943C90608D4F2
:106EF0008168C943C90604D4102141602046FFF7C8
:106F0000B8FE20680168C943890608D48168C9436E
:106F1000890604D4202141602046FFF7A9FF20689C
:106F20000168C943490608D48168C943490604D4A5
:106F3000402141602046FFF79AFF10BDF8B50400DC
:106F400005D025462035A87B002802D006E0012088
:106F5000F8BD00206873204600F04EF80220A873A8
:106F60002068C26884466368012B01D106208243F1
:106F700016486169814202D0072040038243002BFA
:106F800001D1D82082431248A668024018463043F7
:106F9000676A266A3E433043A66A30431043002B9B
:106FA00002D0012B04D005E02369E2691A4300E016
:106FB000E2681043054A914202D0A2691143084396
:106FC0006146C8600120A8730020F8BDFFFF0000E3
:106FD000F8F119FF10B500680549884207D1054846
:106FE000816B4900490881630D2000F073F810BDE2
:106FF000007C00400010024010B50068084988423B
:107000000CD10848816BC204114381630022012125
:107010000D2000F07BF80D2000F06CF810BD000092
:10702000007C0040001002400068C069704700000A
:10703000F8B504460220254620351746A8731D489A
:107040000268C3041A4302602068C2689B121A4394
:10705000C260206802690126324302612268102062
:107060005060206881611021204601F05DFC0328FA
:107070001FD0216808204860206847610821204609
:1070800001F052FC032814D0204601F0DDFBA87B60
:1070900003280ED02068816831438160206801692F
:1070A0003143016120680169042211430161AE731B
:1070B0000020F8BD00040140704700000448416B07
:1070C000012211434163816B0204114381637047C4
:1070D00000100240002809DBC106C90E01208840CB
:1070E00003490860BFF34F8FBFF36F8F70470000F5
:1070F00080E100E0002805DBC106C90E01208840C0
:10710000014908607047000000E100E010B503F09D
:10711000C3FA10BD02494A6882434A6070470000C2
:1071200000700040024801688215114301607047F9
:107130000070004002494A6802434A6070470000FC
:1071400000700040054801680222114301600448B4
:10715000016904221143016130BF70470070004093
:1071600000ED00E0F0B5154A1368154D54152D6A71
:107170002340ED07ED0F002B04D0002D02D0166840
:10718000A64316601668B608B600064316600D489A
:10719000076904263743076101290DD040BF20BF8E
:1071A00020BF0169B1430161002B04D0002D02D042
:1071B000106820431060F0BD30BFF2E7007000405F
:1071C0000000014000ED00E0F8B50446007800271B
:1071D000534D800671D5524E403EB06BC00004D472
:1071E000B06BA9050843B06301274E480168C90583
:1071F00011D40168821511430160FFF7F5FC00907E
:1072000005E0FFF7F1FC0099401A642837D845489B
:107210000068C005F5D532680321090560680A4099
:107220000140914208D08103890F032904D13168BC
:10723000890301D50120F8BD2A69032109040A4008
:1072400022D0084090421FD0207880061CD52869A3
:107250002A6988430121C9040A432A612A698A43A9
:107260002A612861C0050FD5FFF7BEFC009008E039
:10727000FFF7BAFC0099411A2B48814201D903203B
:10728000F8BD28698005F3D561688803800F03285D
:1072900005D132680005824301400A433260286903
:1072A000032261681204114008432861002F04D0B2
:1072B000B16B012000078143B1632078C00705D07E
:1072C000E868A168800880000843E86020788007AB
:1072D00005D5E8680C218843E1680843E860207818
:1072E000400706D5E86803218902884321690843DD
:1072F000E8602078000706D5E86803210903884381
:1073000061690843E8602078000606D5E868032133
:1073100089048843A1690843E8600020F8BD0000A3
:10732000401002400070004088130000F8B50E467F
:10733000050038D05E480068C007C00FB04214D2C4
:107340005B4C20684008400030432060FFF74CFC55
:10735000074605E0FFF748FCC11B564881427AD832
:107360002068C007C00FB042F4D12878524C800783
:1073700005D5E068F0218843A9680843E0602878D3
:10738000C00752D06868022806D0032807D02168B9
:1073900001280AD0890504E02168890301E02168F9
:1073A0008901002903DB0120F8BD4907F9E7E168FD
:1073B000890889000143E160FFF716FC0746686809
:1073C00002280AD0032814D001281ED029E0FFF794
:1073D0000BFCC11B374881423DD8E0680007800F95
:1073E0000228F4D121E0FFF7FFFBC11B31488142A5
:1073F00031D8E0680007800F0328F4D115E0FFF7CB
:10740000F3FBC11B2B48814225D8E0680007800FA1
:107410000128F4D109E0FFF7E7FBC11B25488142B1
:1074200019D8E0680007800FF5D121480168C90725
:10743000C90FB14217D901684908490031430160B9
:10744000FFF7D2FB074608E005E0FFF7CDFBC11BC5
:107450001848814201D90320F8BD15480068C007CB
:10746000C00FB042F1D12878400706D5E068072167
:1074700009028843E9680843E0602878000707D5D7
:10748000E0680721C90288432969C9000843E06010
:1074900000F03AF8E168094A0906090F515CC84052
:1074A0000749086007480068FFF7C0FBF8BD000007
:1074B0000020024088130000001002403EC6000871
:1074C0004801002040010020044805490068C968BF
:1074D000044A4905490F515CC840704748010020E3
:1074E0000010024057C60008044805490068C968F2
:1074F000044A8904490F515CC84070474801002084
:107500000010024057C6000870B51A4AD3681A49DD
:107510000C2018408D0004280CD04E00082810D0F4
:107520000C2810D050680004410F0120C003491CF2
:10753000884070BD1068C00601D5084670BD284659
:1075400070BD304670BD98020C4C000F205C1B02D1
:107550009C0FD368641CDB0301D5314603E012683D
:10756000D20600D4294603F05CF822460023FDF73A
:10757000D5FD70BD0010024000093D004EC6000858
:10758000FEB505007ED0FE4CE7680C20E66807409B
:107590000120000406402878C00747D0082F05D0F6
:1075A0000C2F0AD101200004864206D120688003F6
:1075B0003CD568680028E5D038E0012069680004FF
:1075C000814203D121680143216011E0052301229A
:1075D0001B0492049942216802D111432160F1E712
:1075E0008143216021680140009120689043206020
:1075F000686800280DD0FFF7F7FA009005E0FFF764
:10760000F3FA0099401A64287BD820688003F6D5E5
:107610000CE0FFF7E9FA009005E0FFF7E5FA0099C2
:10762000401A6428F0D820688003F6D428788007B0
:1076300056D50923E868042F0DD00C2F01D1002E58
:1076400009D000283CD02168994301432160FFF70D
:10765000CBFA064628E02168490701D5002891D0D9
:1076600061681F22120291432A691202114361606C
:107670002168994301432160FFF746FFE16809064D
:107680000A0F00E08BE1BF49895CC840BE49086031
:10769000BE480068FFF7CAFA002873D120E0FFF760
:1076A000A3FA801B0228AFD820684007F7D560688E
:1076B0001F210902884329690902084360600FE01D
:1076C0002068400840002060FFF78EFA064604E07C
:1076D000FFF78AFA801B022896D820684007F7D463
:1076E0002878C00660D5002F0CD0A86900284AD0A1
:1076F0002068FF21013108432060FFF775FA064634
:107700002EE0C1E02068800502D5A8690028A6D037
:107710006068072149038843296A084360606068FC
:10772000297F0002000A090608436060286A410BAD
:107730000120C003491C8840E16809060A0F9149ED
:10774000895CC8409049086090480068FFF76EFA6D
:10775000002817D128E0FFF747FA801B0228A2D89B
:1077600020688005F7D56068072149038843296AA6
:10777000084360606068297F0002000A0906084328
:10778000606011E0E2E02168FF2001308143216068
:10779000FFF72AFA064604E0FFF726FA801B0228C4
:1077A00072D820688005F7D42878794E000724D550
:1077B00068690028306910D0012108433061FFF763
:1077C00013FA009005E0FFF70FFA0099401A02281B
:1077D0005AD830698007F6D50FE040084000306184
:1077E000FFF702FA009005E0FFF7FEF90099401A52
:1077F000022849D830698007F6D42878400766D532
:1078000000200290A06BC00006D4A06B01210907E4
:107810000843A063012002905E480168C90511D4A5
:107820000168821511430160FFF7DEF9009005E061
:10783000FFF7DAF90099401A642825D855480068FE
:10784000C005F5D5FF20AA680130824203D1316915
:107850000143316111E001218902002A07D005238B
:107860001B029A4203D132690A433261EFE732695F
:1078700082433261306988433061A868002810D0A3
:10788000FFF7B2F9009008E05FE0FFF7ADF90146BD
:107890000098091A4048814257D830698005F4D5CC
:1078A0000DE0FFF7A1F9009006E0FFF79DF90099C0
:1078B000411A3948814248D830698005F5D4029888
:1078C000002804D0A06B012109078843A063686ADF
:1078D000002866D00C2F3ED00126360602282068EC
:1078E00005D0B0432060FFF77FF905462FE0B04395
:1078F0002060FFF779F9074604E0FFF775F9C01B30
:10790000022822D820688001F7D4E96AA86AE268D0
:107910000843296BFD231B049A4311430843E0608D
:10792000206830432060FFF75FF9054604E0FFF769
:107930005BF9401B022808D820688001F7D530E0A9
:10794000FFF752F9401B022801D90320FEBD206831
:107950008001F5D425E00128F8D0E0680121090470
:10796000AA6A014091421AD10F218904EA6A0140B2
:10797000914214D1032189050840296B88420DE00A
:10798000001002403EC600084801002040010020CF
:1079900040100240007000408813000001D0012018
:1079A000FEBD0020FEBDF8B504000ED0FF27606AC2
:1079B0000537002500280AD0256165612646403636
:1079C000A562707C002807D00AE00120F8BD60683D
:1079D000B842F3D0E561F1E73574204600F03EF897
:1079E000022171742068026840239A4302602123B7
:1079F000A26860689B021A4038401043E3688A021C
:107A00001340184323690B40217D1843C907C90F50
:107A10000843A169931019400843E16938231940CC
:107A20000843216A802319400843A16A9300194042
:107A3000084321680860A0690421000C0840616ABD
:107A4000102319400843216848602068C1699143A8
:107A5000C1616565012070740020F8BD10B586B065
:107A6000044614216846FDF7A2FB104920688842AD
:107A700019D10F48416B821411434163C16A01223D
:107A80001143C162C06A002110400590E0200090BF
:107A90000220019003200390029104910520694681
:107AA0000007FEF7D1FF06B010BD00000030014016
:107AB00000100240094910B5401E884201D901203A
:107AC00010BD074C60610321081F02F0E5FD002096
:107AD000A06107202061002010BD0000FFFFFF0013
:107AE00000E000E0F0B502462032137E012B1ED0EC
:107AF000012515760223537606687468B3687027EB
:107B0000BC430F68274377600068AC07A04205D0EC
:107B1000084CA04202D0084CA04204D180244968FD
:107B2000A34319438160557600201076F0BD0220F2
:107B3000F0BD0000000801400014014070B50500D0
:107B400005D02C462034607E002802D006E00120BB
:107B500070BD00202076284600F010F802206076E4
:107B6000291D286801F0C0FF0120A077A076E076EB
:107B7000207760776076002070BD000000680121EA
:107B80008907884204D10348816B01221143816334
:107B90007047000000100240F8B505460446203545
:107BA000287E012817D001262E76022068762268CA
:107BB00090687727FF23B8431B02984390600A68B8
:107BC000502A31D00EDC202A4BD006DC002A48D0C7
:107BD000102A3AD145E00220F8BD302A41D0402A8F
:107BE00033D136E0602A27D0702A12D0012000035A
:107BF000121A2AD0824228D1CB684A688968206844
:107C000001F0ABFF2068816801229203114381607B
:107C10001BE0CB684A688968206801F09EFF2168F4
:107C200088683843886010E0CA684968206802F0B4
:107C30000EF85021206806E0CA684968206802F002
:107C400017F86021206801F093FF6E7600202876F7
:107C5000F8BDCA684968206801F0F9FF4021206832
:107C6000F1E711462068EEE710B586B0044614210E
:107C70006846FDF79CFA012120688907884212D1E5
:107C80000A49CA6A02200243CA62C96A01900140D5
:107C900005914102009100210291039104906946EF
:107CA0000348FEF7D1FE06B010BD000000100240F0
:107CB00000040050F8B5064604462036307E0D46D6
:107CC00001280BD0012008273076002A08D0042A8A
:107CD00016D0082A2AD00C2A4DD137E00220F8BD50
:107CE000206801F04DFF2068816939438161206877
:107CF000816904229143816120688169EA6812E008
:107D0000206801F055FF206881690122D2021143E9
:107D1000816120688269012189028A438261206829
:107D20008169EA6812021143816124E0206801F050
:107D300058FF2068C1693943C1612068C1690422C4
:107D40009143C1612068C169EA6812E0206801F0CE
:107D500063FF2068C1690122D2021143C16120681A
:107D6000C269012189028A43C2612068C169EA6847
:107D700012021143C16100203076F8BD70B50500D4
:107D800005D02C462034607E002802D006E0012079
:107D900070BD00202076284600F00FF802206076A3
:107DA000291D286801F0A0FE0120A077A076E076CA
:107DB000207760776076002070BD704770B505460B
:107DC0002C4602202034002908D004290BD0082991
:107DD0000ED0627F012A10D0012070BDA27E012A40
:107DE000FAD1A0760AE0E27E012AF5D1E07605E03C
:107DF000227F012AF0D1207700E0607701222868F5
:107E000001F09EFE0122286892070121904205D0D0
:107E1000074A904202D0074A904204D18268520732
:107E2000520F062A02D002680A430260002070BD89
:107E3000000801400014014070B504460D4600687A
:107E4000002201F07DFE2068016A0C4A114203D134
:107E5000016849084900016001202034002D06D046
:107E6000042D06D0082D06D06077002070BDA076C6
:107E7000FBE7E076F9E72077F7E700001111000053
:107E80007047704770470000F8B502680446D06933
:107E900011689668814B05461D402023002D6CD04B
:107EA000F7077F4DFF0FBC460D402F4379D0254685
:107EB000C7078035002F06D0CF0504D501271762EC
:107EC0002A683A432A60820708D5F20706D0276855
:107ED00002223A622A6804273A432A60420708D5F8
:107EE000F20706D02668042232622A68022632434C
:107EF0002A6002070AD50A461A406646324305D070
:107F00002668082232622E6816432E60020508D5C4
:107F10004A0106D501222668D20232622A681A4333
:107F20002A602A68002A30D0800606D5880604D543
:107F3000616E002901D02046884728682168896839
:107F4000490602D42821084225D0204602F0AFF885
:107F500020688168490619D5826840218A43826079
:107F6000206F002812D04F498163206FFEF7D2FBAB
:107F700000280AD0206F816B06E0850611D58D069A
:107F80000FD5616E77E020468847F8BD2046FFF7A1
:107F900079FFF8BD05E02046FFF774FF0020286058
:107FA000F7E7256E012D56D1C50654D5CD0652D51D
:107FB000102616622068816825464906403500294A
:107FC0002ADA226F116849680904090CE1D02F8B65
:107FD0008F42DED9698311680968890617D4016860
:107FE000320191430160206881684908490081603D
:107FF00020688168402291438160E3670020206609
:1080000020680168B1430160206FFEF761FB288B97
:10801000698B401A81B21AE0298B6A8B891A6A8BA4
:1080200089B2002AB5D00029B3D00268FF252135D6
:10803000AA43026020688268520852008260E367A7
:1080400000202066606620680268B2430260204615
:10805000FFF716FF9DE7C50208D5750206D501207A
:10806000000510622046FFF70CFF92E7050605D5D4
:108070000D0603D5A16E002985D18AE7400688D573
:10808000480686D5116820464024A14311608367C5
:108090000021816600F043F97BE700000F08000033
:1080A00020010004D59F000810B5040003D0A06F84
:1080B000002802D007E0012010BD002174200155E6
:1080C000204600F027F82420A067206801684908AE
:1080D00049000160204602F03DF80128ECD0606ABA
:1080E000002802D0204601F055FE20684168092290
:1080F000D20291434160206881682A2291438160C5
:1081000020680168012211430160204601F0A8FEA9
:1081100010BD0000F0B587B0064614216846FDF793
:1081200046F82C493068884251D12B48416B0122D6
:10813000920311434163C16A01221143C162C06AC3
:1081400000251040059003204002009002200327E4
:1081500001A9A1C104200490052069460007FEF78B
:1081600073FC1F4C1D48A560E56081C48027E56055
:10817000A7602020256160610002A0611848083CCA
:10818000FEF742FB002801D0FDF72AFE3467A66205
:10819000144C1248214614382060032060601020DF
:1081A0000831A1C16561A561E56120462562FEF740
:1081B0002BFB002801D0FDF713FEF46600220121FD
:1081C0001B20A662FEF7A2FF1B20FEF793FF07B05D
:1081D000F0BD0000003801400010024030000240B5
:1081E000301600207816002070B5C36F202B27D1E1
:1081F00000290BD0002A09D0012483682403A3425C
:1082000006D10369002B03D1CB0701D0012070BD3B
:10821000034660331C7D012C12D001241C75002301
:108220000366084C0368A34207D05C68240204D5A7
:108230001C680125AD062C431C6002F08BF870BD54
:10824000022070BD0048004070477047FFB50446EB
:10825000806F83B017460D4620285ED1002D0AD0CE
:10826000002F08D0A168C001814207D120690028F1
:1082700004D1E80702D0012007B0F0BD20466030ED
:108280000090007D012848D0009801210175002050
:10829000802108512120A067FEF7A6FC2646403623
:1082A0000190378277820120A1680003814202D1C8
:1082B0002069002805D02F46002500990020087568
:1082C00011E00027F9E700228021204602F088F81B
:1082D000002815D1002F15D02168387888627F1CBE
:1082E000708A401E7082708A019B00280698009058
:1082F000E9D100224021204602F072F8002808D07F
:108300000320B9E728882168C005C00D8862AD1C2C
:10831000E6E72020A0670020AEE70220ACE7704728
:10832000034D044C04A002F05BF9E560FAE700009D
:108330000400FA0500ED00E0486172644661756C66
:10834000745F48616E646C65722E0D0A0000000057
:1083500030B585B014216846FCF729FF1148418BE0
:10836000002901D10221418388B2012807D00228C7
:1083700003D100F003FCFDF755FC05B030BD012230
:10838000094D940221462846FEF727FC00210120D2
:10839000029103910190009469462846FEF754FB30
:1083A000EBE70000F40000200004005010B50524A5
:1083B0002407002204212046FEF70FFC002208219A
:1083C0002046FEF70AFC0A2002F06FFB012204217E
:1083D0002046FEF702FC0A2002F067FB002204217F
:1083E0002046FEF7FAFB10BD10B505242407002235
:1083F00004212046FEF7F1FB012208212046FEF76A
:10840000ECFB0A2002F051FB012204212046FEF77A
:10841000E4FB0A2002F049FB002204212046FEF77B
:10842000DCFB10BDF8B500240526074625463607B7
:10843000002204213046FEF7D0FB0A2002F035FB73
:10844000012204213046FEF7C8FB6006040E082115
:108450003046FEF7B5FB002801D0641CE4B20520CD
:1084600002F023FB6D1CEDB2082DE1D3002F03D0E9
:10847000FFF79CFF2046F8BDFFF7B6FFFAE770B59F
:10848000052605463607002204213046FEF7A5FBE7
:108490000024E80901D0012200E000220821304632
:1084A000FEF79BFB6806050E0A2002F0FEFA012289
:1084B00004213046FEF791FB0A2002F0F6FA002272
:1084C00004213046FEF789FB0A2002F0EEFA641C14
:1084D000E4B2082CDDD370BD10B5052424070122B9
:1084E00008212046FEF779FB012204212046FEF7F1
:1084F00074FB002208212046FEF76FFB0A2002F0E1
:10850000D4FA002204212046FEF767FB10BD10B507
:1085100005242407002204212046FEF75EFB0022EA
:1085200008212046FEF759FB0A2002F0BEFA01227C
:1085300004212046FEF751FB012208212046FEF7C8
:108540004CFB0A2002F0B1FA10BD70B505252D07CD
:108550000024012208212846FEF73FFB062002F0F6
:10856000A4FA012204212846FEF737FB062002F078
:108570009CFA07E0641CE4B2FA2C03D9FFF7C7FFAA
:10858000012070BD08212846FEF71AFB0028F1D112
:10859000002204212846FEF720FB002070BD0000C9
:1085A000F8B501F08FFC01F0C9FC58480068C069BB
:1085B000FDF706FD564C5749A082898F564E00257F
:1085C000002931D0A26A730354499A4202DB022285
:1085D0000A7000E00D700A7801218902002A05D096
:1085E000012A0ED0022A10D0032A1DD1608B012847
:1085F0002BD0022818D1454808214038FFF71CFC31
:1086000012E0FF22F5329042F0D2608B01281AD09E
:10861000022804D008E03046FEF7DFFA04E03B48C9
:1086200008214038FFF7CAFB0121C9023046FEF796
:10863000C7FA0127FF0300282AD039480560E079EE
:10864000002804D007E00022E5E70122E3E701204B
:10865000E07101F027FF2078632806D90022082165
:108660003046FEF7BAFA012205E001220821304621
:10867000FEF7B3FA0022052039460007FEF7ADFAEF
:10868000244C284E4034A08C274F012803D01CE0F6
:10869000E5710022EAE725486946088072B6802124
:1086A0002348FDF7B5FB002804D002226946204884
:1086B000FDF752FC62B61FA001F092FFA58403F003
:1086C000D1FE642002F0EAF9FE60608C012808D136
:1086D00010486584058003F0C5FE642002F0DEF9D1
:1086E000FE60208C012806D1258403F0BBFE6420A7
:1086F00002F0D4F9FE600748124A0188914202D183
:10870000C088002800D1FE60F8BD0000AC15002034
:10871000F4000020AC0D0020000400508100002077
:10872000380100200400FA0500ED00E0AAAA0000CC
:10873000384A0008BDF8C8EBC9FDBCB6C4A3CABD21
:108740000D0A0000AA55000008B53721202000F0CE
:108750006EF80321212000F06AF84021222000F069
:1087600066F80821232000F062F8AA21302000F0EA
:108770005EF80A48008FC1B2322000F058F802219A
:10878000332000F054F85F21202000F050F86846B4
:1087900000F006F80A2002F088F908BDAC0D0020B0
:1087A00010B501460F2000F021F8002800D001206C
:1087B00010BD10B50446FFF78FFE3220FFF75FFEB5
:1087C000FFF7C3FEE0B2FFF75AFEFFF7BEFEFFF76A
:1087D00083FE3320FFF753FEFFF7B7FE0020FFF7BD
:1087E00021FE0446FFF793FE204610BD10B50C464F
:1087F000FFF7DFFF2070012010BD70B50D46044665
:10880000FFF76AFE3220FFF73AFEFFF79EFEE0B266
:10881000FFF735FEFFF799FE2846FFF730FEFFF71A
:1088200094FEFFF774FE0A2002F03FF970BD10B508
:10883000FFF7E3FF012010BD10B50248FEF719FB5A
:1088400010BD0000E4140020FEB50446002772B6F7
:10885000334A01688B1804D13248C768032080046A
:10886000074088680190C868009048698E69002BAD
:1088700008D12C4940398B6ACD042B438B628B6A1B
:10888000AB438B62014631433CD025492368CB4240
:1088900005D12449CA6803239B049A43CA6025462C
:1088A0002035002810D021680A6901231A430A6183
:1088B000216848610821204600F036F8032800D1DD
:1088C000A873216808204860002E10D02068016934
:1088D000012211430161206886611021204600F0C9
:1088E00023F8032800D1A8732168102048600C48A1
:1088F0002168C14206D10B48C1680322920491430A
:108900003943C16020680169490849000161216853
:108910000198886021680098C86062B6FEBD0000BA
:108920000084FFBF4010024070B506460B480D465C
:10893000002409490068FCF7DBFB7D21C90048439E
:108940003168401E00D103240B682A469A4301D0A7
:108950000028F6D1204670BD204E000048010020BE
:108960001CB5002116480091144A01910260C163B0
:108970001205426081600722826301220261024681
:10898000C16020321170FF235170C2334362816293
:10899000117301638161042241634261C161FDF78A
:1089A000FDFC084800908013019069460448FDF7DB
:1089B000A5FC00210248FDF74BFC1CBD0024014032
:1089C000881400200200000408B50848016B012249
:1089D00011430163006B01211040009000220A2026
:1089E000FEF794FB0A20FEF785FB08BD001002404D
:1089F000F0B587B014216846FCF7D9FB4748C26A36
:108A000004210A43C262C26A0A400592C16A8026F2
:108A10003143C162C16A31400591C16A01242143D9
:108A2000C162C16A21400591C16A02252943C16220
:108A3000C06A22462840059005201C210007FEF749
:108A4000CCF8012236493748FEF7C7F800223649EC
:108A50003448FEF7C2F891210520002209020007E0
:108A6000FEF7BBF8314801900027052069460297C0
:108A700000940007FDF7E8FF0C2000901120019002
:108A8000032003900520029769460007FDF7DCFFED
:108A900010206A46039591C2052069460007FDF73C
:108AA000D3FF1120019002976946039700941D4857
:108AB000FDF7CAFF1E4801906946009502941948C7
:108AC000FDF7C2FFE0020090694601970295154844
:108AD000FDF7BAFF1748694691C1694611480397E7
:108AE000FDF7B2FF91200002694691C10520694659
:108AF00000070397FDF7A8FF69460A48019700960B
:108B00000294FDF7A1FF002201210520FEF7FEFAE5
:108B10000520FEF7EFFA07B0F0BD0000001002409C
:108B20000102000000040050083000000000111095
:108B3000000021100832000010B50F4C0D482060D5
:108B4000FF20053060600020A060E060206160616F
:108B5000E0610121206249026062A161A0620720F8
:108B6000E0622046FEF71FFF2068016840221143A3
:108B7000016010BD003001401415002010B58AB00E
:108B8000002404940594069407940894012118483D
:108B900009940094019402948907039401600921C7
:108BA00084604160046113494461C160FEF7C6FFFF
:108BB00001200003049004A90D48FEF7EDFF0C48C6
:108BC000FFF7DCF8089408A909480994FEF78AFF22
:108BD000602000900848019002940822694603949E
:108BE0000348FFF767F80248FFF73EF80AB010BDE8
:108BF0006C150020930400005702000000B585B0FA
:108C000014216846FCF7D3FA0E480D490160E121B2
:108C10004902416000218160C160016181610C22D3
:108C2000C161426101623021416201210903816316
:108C30004900C163FFF738FA01F02EFC05B000BD12
:108C400000380140AC15002070470000F0B589B035
:108C50000A2002F075FC7D20C00002F08BFCFF4C66
:108C60000020A070FE492165617B0C2901D30B21F6
:108C700061730025FB48E570FB4E00783071FB49BD
:108C8000A079097840000843E17C89000843F0712D
:108C9000E06AF070010A3172401CE062607931468E
:108CA000B0744200B4310846A138FCF767FA607925
:108CB000EF498200400080191330121DFCF75EFA64
:108CC000EC48218D008940182085607906214843B1
:108CD000E249821920310B7AD375497A117606213F
:108CE0007172E5491C300978B172A17E3173314649
:108CF0001339227F0A75627F4A750022133102F010
:108D000009FD60790621484300211C3002F014FD62
:108D1000022002F065FCF571E573A5720126267349
:108D2000E572D648FEF780F920840746E570607941
:108D3000FCF704FDD24AD34BFCF7E4FB01F04AFEFA
:108D40000022B307FCF72CFBFCF758FD0006C00C13
:108D5000C01980B2F1036084884201D3401A608454
:108D6000C948E0632079401C2071C448FEF75CF9D3
:108D7000E083BD480C300546423540300390C1E1E8
:108D8000BE48FEF751F9E083C04F0BE0BB48FEF749
:108D90004BF980B2E083618C884203D3BC4A8918C6
:108DA000884206D300210F2002F04AFB384220639C
:108DB000ECD0206B411C21D040047CD58122D20113
:108DC00000210F2002F07BFC7D20C00002F0D2FBCE
:108DD000002002F084FB0021102002F031FB41064C
:108DE000A148490E274600225030E16402F05EFBA4
:108DF0009D485030417A0729C1D101E001F06EFC55
:108E00000222A449401DFCF7DDF90028B7D102F089
:108E1000E4FCF965B86502F0CDFC79663866F8784F
:108E20006A46401CF87090484D30017911704079C5
:108E3000507010880490B98B88427DD1964F288A53
:108E400038800398808A20838C48FEF7EDF8E08311
:108E500002F008FAFF22216E5204606E0023891886
:108E600058410206080A1043009040084000010ED5
:108E70000002E166A0667C48E36D0A30A26D02F054
:108E800081FC6079636E81007748226E0818163085
:108E900002F078FC7448E36E1230A26E02F072FCAD
:108EA000714808214172A07C002816D06E48022229
:108EB0007849553000E018E1FCF784F900280CD11E
:108EC0006948E673C671E06C67491638C2B266310C
:108ED00008462274EA30FCF751F9607900228000DC
:108EE00061491C3002F016FC6079002180001C30C2
:108EF00002F022FC009802F01CFB012002F070FB43
:108F0000207202216548FDF75BFE00287ED000211B
:108F10005648574B01705148A9890187EA89428711
:108F2000A06BE06318601846C438C37C1807000FB4
:108F3000032800D0607400E078E01809A0740020D5
:108F40002071464BA6729987DA87E672218B544AC4
:108F5000FF31C33189B2218391420BD95242891822
:108F6000218339887D22491C89B2D20039809142FF
:108F700000D338803D887D20C000218B6843401895
:108F8000206407904748302107784748A773008836
:108F90004843FCF7B8FB02900A2029464143608B06
:108FA000302206905043081AFCF7A2FB0299FCF706
:108FB000ACF97F21C905FCF712F9FCF7E6FB80B29A
:108FC00038497F1E0880B84200D1E672A58414207B
:108FD000205EFCF79FFB07460391E08BFCF7AEFB9E
:108FE000324A334BFCF78EFA05460E460798FCF7DB
:108FF00091FB2A463346FCF777FA3A46039BFCF787
:10900000CFF9FCF7D7FB6064069800E005E000F0BC
:10901000A3FC207A002802D07DE0012178E700211E
:109020000F2002F00DFA0006F9D574E0FCF7B0FF4E
:109030000F4A0321303211540849AA890A87EA8964
:109040004A870B4980003039421803990190098BF7
:1090500011800749BA6B41184A602BE0700000206C
:109060003F420F00F40000202012002034010020B5
:1090700034130020AC0D002004010020E414002073
:10908000B81E85EB51B8CE3FA086010000D0272442
:10909000983A000018010020300100200004005020
:1090A000E70300001001002014010020F853E3A59D
:1090B0009B843E4041497B6E401816303A6E02F068
:1090C00061FB396DB86B884200DA38653B4A01991B
:1090D000E4325158814215DD002913D0002811DDFA
:1090E0000498B883022038700CE03A4600210F2023
:1090F00002F0E5FA6079E178401C814202D000205C
:1091000002F0EDF9E08B618C884200D238E62C4AFF
:1091100089188842FAD8A07A012801D00220A072CA
:1091200002F0A0F8274A00210F2002F0C8FA2079A7
:10913000002807D024490A2209885143814201D2DC
:1091400000202070E07B00281DD020490B78487853
:109150008A78022B17D110280CD0C82813D21C4BA8
:10916000C91C1818FCF70AF803F07CF9642001F018
:1091700095FC43E6174D28684000000E03D1C878DF
:10918000FCF7C1FA2860114D00209C3D2E46217845
:109190006379183607E04200AF5AB25A974200D0BE
:1091A0000221401CC0B29842F5D3064A2170803299
:1091B00000210F2002F083FA09B0F0BD2012002038
:1091C000983A000000D027240401002070130020EA
:1091D000AC0D00201C01002070470000F0B58DB0E0
:1091E000B44801900020C0430A9000260A2002F0F3
:1091F000A7F97D20C00002F0BDF90020AE4C054665
:10920000A070AE4FAE480B90AD480022C2388573B7
:109210000146142002F07EFA0021142002F08CFA9C
:10922000022002F0DDF900210F2002F009F9384296
:109230002063F8D0206B411C18D040047ED58122D9
:10924000D20100210F2002F03AFA0021102002F092
:10925000F7F841069A48490E0022801C02F026F9D0
:109260009748801C417A022902D007E101F036FAC2
:10927000934802229349C01DFBF7A4FF0028F4D1B4
:1092800002F0ABFAE165A06502F094FA616620662F
:10929000002E22D10B988C49008A0880884801262C
:1092A000801E808A20838948FDF7BEFEE083208BE4
:1092B0008749FF30C33080B2208388420DD94942AC
:1092C0004018814920830888814A401C80B20B32B3
:1092D0000880904201D3002008800B9968468A8953
:1092E0000280C989418076490422C91C0846A238F7
:1092F000FBF744FFFF22216E5204606E00238918A1
:1093000058410006090A01430846029102F011F98A
:10931000029948084000010E0002E166A066684814
:10932000E36D9638A26D02F02DFA6548636E9238AF
:10933000226E02F027FA62488E3800E0A0E0E36E69
:10934000A26E02F01FFA5E490022A0393C2002F012
:10935000E1F900213C2002F0EFF9012002F040F990
:109360002072A0780121401CA0700520C9030007CD
:10937000FCF722FE54487D220088D200014602906C
:109380005043228B0A39801820640C905148007891
:10939000A073049008B2E084002803DA7D21C9009C
:1093A0004018E0844C48302100884843FCF7ABF972
:1093B00005902620205EFCF79BF90599FBF7A5FF99
:1093C0007F21C905FBF70BFFFCF7DFF9414980B2AC
:1093D00008800499491E884201D10120E072029858
:1093E000A0841420205EFCF795F905910690E08B8F
:1093F000FCF7A4F9394A3A4BFCF784F8079104903A
:109400000C98FCF787F9079B049AFCF76DF8059B0D
:10941000069AFBF7C5FFFCF7CDF96064608B00F09E
:109420009BFA00990198814210DA00290ED0244954
:109430000422C91C0AA8FBF7A1FE022020702948BB
:109440000A2100784843607200980190207A002831
:1094500005D100210F2001F0F3FF0006F9D580228D
:1094600000210F2002F02BF900206D1CEDB260707E
:10947000032D00D2C8E6002E08D017E00120F4E743
:10948000194A00210F2002F01AF9F7E7618B1748FB
:10949000002902D00288914201D90188618388B2F3
:1094A0001349401E09884843124908800A98A0833E
:1094B0000DB0F0BD3F420F007000002000D0272407
:1094C0006E1200201801002030010020E41400205A
:1094D000E70300001001002014010020F853E3A569
:1094E0009B843E40040100200090272400010020BE
:1094F000FE000020FC000020F8B531492F4808602C
:1095000002F054FA2F4800F0E7F92F4CE0822D4882
:10951000801C00F0E1F920832A48001D00F0DCF9EE
:1095200060832B4829494180014640310979294F00
:109530000906090E617006D1C7800121C1870A2181
:10954000418700218187244AC18E1170C18F6171CA
:10955000818FA171817AE1708588052165626181C1
:10956000C6883046FBF7C4FDA08101462846FBF7BC
:10957000BFFD8800081885B2164825816843FCF7AE
:10958000DDF8164A164BFCF725F8FCF737F9E081B1
:10959000658231463846FBF7ABFD20820146C82084
:1095A000FBF7A6FD20840120A083FCF709FDA08223
:1095B000E2890C490C48FDF73BFDF8BDD1A4000839
:1095C00068000020004F0008F4000020190200008D
:1095D000AC0D0020E803000018000020F853E3A5BC
:1095E0009B843E40FF7F0000E4140020F0B5954DC1
:1095F00085B001202880944FC820944C3880E079B1
:10960000401CE071C00706D0608B411E61830228B8
:1096100001D2C8206083608B00F09EF90A2001F01F
:109620008FFF7D20C00001F0A5FF02218848FDF7D3
:10963000C7FA002838D00020864980000978874E74
:1096400049000843844909780843B07210207072B9
:109650008348C1887D20C000FBF74AFD70738148B4
:109660007F490078B07330460B308A780270C97831
:109670004170411C7A482030027ECA70407E0871D9
:1096800077482230027E4A71407E887100220C3970
:10969000152002F03FF80021152002F04DF80220BD
:1096A00001F09EFF704E03E00120C5E7FEF778FF52
:1096B00000210F2001F0C4FE30422063F6D0206B61
:1096C000411C7DD040047CD58122D20100210F2095
:1096D00001F0F5FF0021102001F0B2FE41065F48C5
:1096E000490E00225030E16401F0E0FE5B4E50363E
:1096F000707A112865D102225C49701DFBF762FD6A
:1097000000285ED1F01E027969460A7040794870DF
:10971000B17A2980C820FBF7EBFC3880307B60836E
:10972000534DB01E008A2880301F808A2083514804
:10973000FDF77AFC80B2E0830390208B4E49FF3026
:10974000C33080B2208388420CD94942401820831C
:1097500028884949401C80B20B312880884201D3B7
:10976000002028802D887D20C000218B6843401870
:10977000206401904148067828460A3800B2A67352
:10978000E084002803DA7D21C9004018E08438888D
:1097900030214843FBF7B7FF07462620205EFBF742
:1097A000A7FF3946FBF7B1FD7F21C905FBF717FD80
:1097B000FBF7EBFF80B23149761E0880B04201E032
:1097C0003EE03BE001D10120E072A5841420205E40
:1097D000FBF7A0FF02900F460398FBF7AFFF284A64
:1097E000284BFBF78FFE05460E460198FBF792FFCC
:1097F0002A463346FBF778FE3B46029AFBF7D0FD3C
:10980000FBF7D8FF606468460088A08313481349BB
:109810005030807C63316071420008460D46513003
:10982000FBF7ACFC6079294642000C48CC30FBF7D2
:10983000A5FC608BFF2801D00320207005B0F0BD8F
:1098400000F04CFF040100201401002070000020F3
:1098500000040050F9000020FA000020201200202F
:10986000AC0D00201800002000D027241801002093
:1098700030010020E4140020E70300001001002064
:10988000F853E3A59B843E4070B586B0142168462A
:10989000FBF78DFC01250F4EED03002229463046D3
:1098A000FDF79BF901200024019002946946009580
:1098B00003943046FDF7C8F80320019002946946EE
:1098C000009503943046FDF7BFF8022001F0E6F85A
:1098D00006B070BD0004005000887047704700005B
:1098E000F8B5044600206A461080194D55222A70AA
:1098F000AA226A700322AA70661DEE702A7169712D
:10990000144A49008918AC712246E81DFBF736FC61
:10991000002007E029186A468978128889186A4663
:109920001180401CB042F5DB611DA81CFCF79EF9BC
:1099300001466846018029190078C8716846407858
:10994000087221460931024800F0D2FBF8BD000040
:1099500024140020AC0D002010B51B4C228A01E01D
:10996000891AA183A18B9142FAD2228C8BB25343E4
:109970001B18E383132902D14A431018E083E08BBC
:1099800030214843642164304843104960630968CA
:10999000401A4B21090140182063FBF7BBFE0C4A1B
:1099A0000C4BFBF717FEFBF705FF0B49E062884203
:1099B00002DD4A428018E062002801DA4018E062C5
:1099C00006490968486110BDF4000020B400002079
:1099D000F853E3A59B843E40FF7F0000E414002081
:1099E000034A1168382389B29943014311607047D3
:1099F0000030014010B5FDF7FDF810BD10B59AB06C
:109A000034216846FBF7D3FB14210DA8FBF7CFFBED
:109A10001C2112A8FBF7CBFB1B4801680324E402BE
:109A2000A143C21489180160FDF77CFB1748016946
:109A3000A143016106200090FF2001300290012027
:109A40000390102004900220099040040B90000124
:109A500000240C900A946846FDF792FD0F200D90AB
:109A600003200E900F941094012111940DA8FDF77E
:109A70005DFC81201290032080041890149412A899
:109A8000FDF7A2FB1AB010BD00700040401002406C
:109A900010480168821511430160C1680E4A1140E7
:109AA000C16001680D4A11400160816849084900A0
:109AB000816001680122920491430160C168FD2226
:109AC00012049143C1600021016106490448886085
:109AD00070470000001002400C40FF88F6FFF6FEC1
:109AE0000050000800ED00E070B5026801239B07FC
:109AF000114C124D984203D0A04201D0A84203D18C
:109B00007026B2434E683243984203D0A04201D03F
:109B1000A84204D103231B029A43CB681A43802333
:109B20009A430B691A4302608A68C26209688162BB
:109B30000121416170BD0000000801400014014096
:109B400010B5CB06DB0E0121046A99408C430462F8
:109B5000016A9A401143016210BD30B58468FF2547
:109B60002D021B021343AC430B432343836030BDE0
:109B7000826870239A430A4307210A438260704730
:109B800030B5026A520852000262026A456883696F
:109B90007024A3439C080B68A40023430224A2431F
:109BA0008C6845601443836149684163046230BD39
:109BB00030B5026A10239A430262036A45688269DB
:109BC00073242402A2430C682402144320229343EA
:109BD0008A68456012011A438461496881630262A0
:109BE00030BD30B5026AFF2301339A430262026A34
:109BF0004568C3697024A3439C080B68A4002343F1
:109C000001246402A2438C68456024021443C361AA
:109C10004968C163046230BD30B5026A01231B0389
:109C20009A430262036A4568C26973242402A2430C
:109C30000C68240214430122520393438A6845604E
:109C400012031A43C46149680164026230BD30B531
:109C5000036A046A6408640004628469F025AC4302
:109C6000120122430A24A3430B438261036230BDE5
:109C700030B5036A1024A34303628469036A0F2585
:109C80002D031203AC432243A024A343090119432B
:109C90008261016230BD0000F8B5102605252D0750
:109CA000AE62AF20800000F000FFFCF71BFA3048E6
:109CB0002E490068FBF7ECFAFBF74EFD2D4C208592
:109CC000AE6101F0D1FB2C4F2C4E60650EE001F02F
:109CD000CBFB6065FEF764FC606B411C616314287C
:109CE00004D927A000F07CFC2948C760606DB04211
:109CF000EDD10026666320780127FF03002806D0F7
:109D000001280CD0022817D003282BD128E00122EB
:109D100039462846FCF761FFFFF768FC06E00122A0
:109D200039462846FCF759FFFFF758FA0022394612
:109D30002846FCF752FF15E0607A0122401E60724F
:109D400039462846FCF749FFFCF756F90022394608
:109D50002846FCF742FF607A002803D1267001E014
:109D6000FEF774FF01F066FAF8BD00000000C8427B
:109D700000000020700000200400FA053001CADE57
:109D80004457204944204552524F522E0D0A00009C
:109D900000ED00E010B5818CC90707D001684A6862
:109DA00001235B049A43836A1A434A60818C8907C2
:109DB00007D501684A6801231B049A43C36A1A4302
:109DC0004A60818C490707D501684A6801239B04D2
:109DD0009A43036B1A434A60818C090707D50168CF
:109DE0004A680123DB039A43436B1A434A60818C20
:109DF000C90607D50268916801231B039943836B49
:109E000019439160818C890607D501688A6801230E
:109E10005B039A43C36B1A438A60818C490612D54F
:109E200003685A6801210905046C8A4322435A6079
:109E3000026C8A4207D10268516803235B0599438B
:109E4000436C19435160818C090607D501684A6843
:109E50000123DB04806C9A4302434A6010BD00007A
:109E6000F8B50446002680300660FCF7BDFE0546C6
:109E700020680068124F000709D501212B460022F7
:109E800049052046009700F0ABFA00280DD1206864
:109E9000006840070BD501212B460022890520468A
:109EA000009700F09DFA002801D00320F8BD202083
:109EB000A067E0672666603426750020F8BD0000C4
:109EC000FFFFFF01F8B5184CC826E078002829D11B
:109ED0006079002826D101206071144D686B00273D
:109EE00000281ED0686BC821081A15E01048E168E8
:109EF000405C616988470F480A21008848430E4941
:109F00000880E068401CE060E068C82800DBE7608B
:109F1000696BC820401A761EE168814201D0002E8C
:109F2000E4DC6771F8BD000054000020000002402E
:109F3000E40C0020040100201601002070B5224C22
:109F4000E07800283FD1207900283CD10120207101
:109F50001E4EF16900250906002933DA21566257A1
:109F600091420AD1F06940062CD5A079002829D069
:109F7000A5712089401C208124E0A179002903D10A
:109F8000A0710A2000F091FD00202056CC2148430A
:109F90000F494218206912181279B262401C00223F
:109FA0002061A256CC235A43895881420ADC25619C
:109FB0002078401C207020780E2800D12570A078D1
:109FC000401CA070257170BD540000200038014075
:109FD000BC01002010B5806A0022014640314A834E
:109FE0004A82FDF74FFF10BD70B5846AA06FE56F20
:109FF0002168896800260906002906DA212804D18B
:10A0000052200653204600F06BF820688068400616
:10A0100006D5222D04D15A200653204600F047F8D9
:10A020002046803001681022114301602046FDF770
:10A0300029FF70BD10B501460968806A0968890664
:10A040001CD400225A210A5201680A68FF230133F6
:10A050009A430A6001688A68520852008A6001685F
:10A060008A6840239A438A602021C167016E0129D2
:10A0700004D101680A6810239A430A60016E01291D
:10A0800002D0FEF7E1F810BD5821095AFDF7F8FE9D
:10A0900010BD10B5806A016E012902D0FEF7D5F817
:10A0A00010BD5821095A4908FDF7EAFE10BD0168A4
:10A0B0000A68FF2321339A430A6001688A685208BC
:10A0C00052008A60016E012904D101680A681023D8
:10A0D0009A430A602021C1670021016641667047EA
:10A0E00001680A68C0239A430A602021816770478B
:10A0F00070B5164CE278002A0CD12279002A09D1D9
:10A100000122E2700025C82903DC0222A256002A9F
:10A1100001DCE57070BD0123E356CC2253430C4AA9
:10A12000D1500123E356CC2673439B180A460146BF
:10A13000181DFBF723F86078401C607060780E28CB
:10A1400000D16570A078401EA070E2E754000020A6
:10A15000BC010020F8B50446016880682369E669FF
:10A1600018436369002533431843724A0B68724EE3
:10A17000334003430B602168486803231B03984363
:10A18000E368184348602168A069914201D0236ABE
:10A1900018438B680B263602B34303438B60674931
:10A1A000236867488B420CD1C0688007800F06D0B7
:10A1B000012839D0022835D0032821D11EE00127FB
:10A1C0001FE060498B420AD1C0680C21084027D0AB
:10A1D000042829D0082825D00C2811D10EE093425C
:10A1E0000ED1C16803208002014019D001208002F5
:10A1F000091A19D0091A15D0814201D1082700E0A7
:10A2000010274F49504840398600934232D1002FE1
:10A210000CD0022F0DD0042F10D0082F7FD126E0B4
:10A220000027EEE70227ECE70427EAE7FDF74CF901
:10A2300006E00968C90605D4304603E0FDF764F975
:10A24000002872D0626851005118814267D811030A
:10A25000814264D3010E0602500800233018594190
:10A26000FAF75CFF03210902411A384A55E0012040
:10A27000C003E7E70122E369D20393422BD13B00FD
:10A2800000F0E7F90906090C4D114D4D4D274D0021
:10A29000FDF71AF909E0FDF727F906E00968C90694
:10A2A00005D4304603E0FDF72FF900283DD0616862
:10A2B00040004A088018FAF71BFF80B20146244A82
:10A2C000103991422BD8511C01400007400F084320
:10A2D00029E01046EBE73B0000F0BBF90906090C4A
:10A2E0002112212121232100FDF7EEF80AE0FDF7DC
:10A2F000FBF807E00968C90606D4304604E00EE022
:10A30000FDF702F9002810D061684A081018FAF722
:10A31000EFFE80B201460E4A1039914203D9012561
:10A3200003E01046F0E72168C86000206066A06680
:10A330002846F8BD00480040F369FFEF00380140AF
:10A34000401002400044004000093D00FFFC0F00A7
:10A35000EFFF0000F8B5044641654030002627466F
:10A36000028380373E602220E0672546206F6035FB
:10A3700000281CD01749C162216F17480863216F5C
:10A3800016484863206F8663236F606D9C461346B2
:10A390002168024660462431FCF77EFA002806D088
:10A3A000102038602E752020A0670120F8BD2E7582
:10A3B00020680168FF220132114301602068816832
:10A3C000012211438160206881684022114381602D
:10A3D0000020F8BD35A0000893A00008E99F000800
:10A3E000FFB581B005460F46044660350A9E39E048
:10A3F000701C37D0FCF7F8FB0499401AB04222D801
:10A40000002E20D02068016849072BD5C069C043C1
:10A41000000527D401202168C00208622068016875
:10A42000FF22A132914301602068816849084900F8
:10A4300081602020A067E0678034206000202875BC
:10A44000032005B0F0BD20680168FF22A1329143CE
:10A450000160206881684908490081602020A06768
:10A46000E067EBE72068C1693846884305D00021E2
:10A4700003988142BCD00020E3E70121F8E7000007
:10A4800010B504491020096808620248FDF7FCFC79
:10A4900010BD0000AC15002001490D2088707047E8
:10A4A0005400002010B507480A22018A5143418414
:10A4B000FEF78AFAFEF7A2FBC82203490348FDF71C
:10A4C00093FE10BDF4000020E40C0020AC15002029
:10A4D000F8B53E4C002321783D4A1D46082910D08E
:10A4E000072947D0062950D0052952D0042953D036
:10A4F000032954D0002956D0012958D002295AD016
:10A500005BE0A17800264A1F04E0314FBF5DFB18D5
:10A510009BB2761C9642F8DB667927799A19511816
:10A52000E3786278C9188918C9194018C043000631
:10A53000000E1AD1012E14D0022E16D1254824491E
:10A54000C018FAF71BFE01F08DFF642000F0A6FA98
:10A55000BFF34F8F21492048C860BFF34F8F00BF22
:10A56000FDE759081046FFF7BBF92570E570A570A7
:10A57000A571F8BDA1795054491CC8B2A071A17849
:10A58000491F8842F5D1082001E060700720207043
:10A59000F8BDE0700620FAE760710520F7E7A070CB
:10A5A000E5700420F3E7552807D10120EFE7AA283A
:10A5B00003D10220EBE7032803D02570E570A570D6
:10A5C000F8BD032020702071F8BD0000EB000020D2
:10A5D000C0130020AC0D00200400FA0500ED00E0DF
:10A5E00010B5024A024900F0E5F910BD9DB7000818
:10A5F0004C0100202021020C01D010211046020A3B
:10A6000001D010460839020901D01046091F8208FE
:10A6100001D01046891E420801D0881E7047081AD2
:10A620007047F8B5040C8BB2264682B25E430D0C1F
:10A630001046370C584336048019002179411646DC
:10A640006E43370C36048019794126466E438919CA
:10A65000F8BD30B47446641E2578641CAB4200D249
:10A660001D46635D5B00E31830BC18474900CA0211
:10A670000243100000D004204A0D01D001221043F3
:10A68000044A490D914201D102210843012800D119
:10A6900005207047FF0700008307FF22DB0E9A406A
:10A6A0008907090E9940002808DB830809489B00A8
:10A6B0001B18186890430843186070470007000F84
:10A6C0000838830804489B001B18D8699043084346
:10A6D000D861704700E400E000ED00E0BFF34F8F69
:10A6E00004490348C860BFF34F8F00BFFDE7000077
:10A6F0000400FA0500ED00E0F8B504464F1EC8005E
:10A700000838211815461E46086849683A46062347
:10A710009A4310D02A463346FAF7F4FE3A46D2005E
:10A72000083AA3181A687F1E5B68FAF739FE0622FA
:10A730003B469343EED1022F23D0042F11D0062F96
:10A740002FD12A463346FAF7DDFEE36AA26AFAF70A
:10A7500027FE2A463346FAF7D5FE636A226AFAF7DD
:10A760001FFE2A463346FAF7CDFEE369A269FAF7DF
:10A7700017FE2A463346FAF7C5FE63692269FAF7DF
:10A780000FFE2A463346FAF7BDFEE368A268FAF7E1
:10A7900007FE2A463346FAF7B5FE63682268FAF7E1
:10A7A000FFFDF8BD002210B5134610460149FAF727
:10A7B00011FF10BD0000F03F10B5FAF7F1FD10BD1C
:10A7C000002210B5134610461146FAF703FF10BDDC
:10A7D00010B50721024A00200907FAF773FF10BDE0
:10A7E00001030000034A10B500201107FAF76AFFC1
:10A7F00010BD000001FDFFFF02E008C8121F08C1E4
:10A80000002AFAD170477047002001E001C1121FF1
:10A81000002AFBD170470000014908607047000022
:10A820005001002008B50021684601706B460122E6
:10A8300002212C2000F052FF0221684601706B4675
:10A8400001222C2000F04AFF08BD000038B5044664
:10A850006D20694608706B46012207492E2000F0E2
:10A860003DFF0649002C01D0054A00E0054A2E2094
:10A8700000F01AFF38BD00000608000006180000AE
:10A88000070600000716000038B504466B46022292
:10A890000021362000F0EEFDB3212300FFF7D9FEA2
:10A8A0000E0F08153A3A3A3A1C273A3A2F34483AEA
:10A8B00000216846017040784108490014E069466B
:10A8C000087880088000401C04E069460878800809
:10A8D0008000801C08701DE0684602780A404832FB
:10A8E00002704178802001436846417012E068465A
:10A8F00002780A40027040784106490EF4E7694642
:10A9000048780221084303E069464878FD21084061
:10A91000694648706B4601220021362000F0DEFEB9
:10A92000012200AB11463620013300F0D7FE38BDBE
:10A9300069460878CF21084069462030CAE708B543
:10A94000032168464170012101706B4602220021FB
:10A95000362000F0C3FE0122D20306212D2000F094
:10A96000A3FE012000F09AF80120FFF78DFF08BD3B
:10A9700008B5020A69464A7008706B460222042133
:10A980002D2000F0ABFE0320694608706B460122C3
:10A9900006212D2000F0A2FE0020694608706B46BB
:10A9A000012206212D2000F099FE0A212D2000F021
:10A9B00047FD08BDF8B516460F460446002503E0DE
:10A9C0003946B047641C6D1C20780028F8D1284611
:10A9D000F8BD0000F8B54A002B4B520DD6182B4A93
:10A9E0000C460546142E2BDA002E12DA284BFAF705
:10A9F000D7FC00221346FAF733FF40D2002C03DACB
:10AA00000124E40700253AE02046284337D0214CB2
:10AA100014E0214F0B46F7403B402B4331D01C4BF9
:10AA2000FAF7BEFC00221346FAF71AFF27D2002CD1
:10AA300003DD01200005F0400419BC4300251EE0A1
:10AA4000332E1EDC33460027143BFF43DF403842E1
:10AA500017D00F4BFAF74EFD00221346FAF700FF0E
:10AA60000DD2002C0ADD142E0CD03420811B0120C5
:10AA700088404019A84200D2641C0546BD432146C7
:10AA80002846F8BD641CF9E701FCFFFF9C750088AF
:10AA90003CE4377E0000F03FFFFF0F007D2110B542
:10AAA000C900484300F001F810BD002140E000BF9C
:10AAB00000BF00BF00BF00BF00BF00BF00BF00BF9E
:10AAC00000BF00BF00BF00BF00BF00BF00BF00BF8E
:10AAD00000BF00BF00BF00BF00BF00BF00BF00BF7E
:10AAE00000BF00BF00BF00BF00BF00BF00BF00BF6E
:10AAF00000BF00BF00BF00BF00BF00BF00BF00BF5E
:10AB000000BF00BF00BF00BF00BF00BF00BF00BF4D
:10AB100000BF00BF00BF00BF00BF00BF00BF00BF3D
:10AB200000BF00BF00BF00BF00BF00BF00BF491C87
:10AB30008142BCD37047FFB581B01E460F4604006A
:10AB400026D00B9903980143A06A394382680720F5
:10AB50009047002818DB0A99A06A314382680620D2
:10AB60009047002810DB25462035A979032F01D90D
:10AB700008200143032E01D904200143A06A826802
:10AB800009209047002806DA0120C04305B0F0BD37
:10AB90000020C043FAE7384600F000F92060304654
:10ABA00000F0FCF860600A9868700398A870EF7075
:10ABB0002E710B9868710020E8E70000F7B5044695
:10ABC000002090B000900190002C05D06A4606212C
:10ABD00001F082FC062803DA0020C04313B0F0BD68
:10ABE0006846407801026846007800040918684603
:10ABF00080780818FAF7A2FD0546684603910079A7
:10AC000001026846C07800040918684640790818AF
:10AC1000FAF794FD032206460F4692075C4BFAF7BB
:10AC20001FFE07D200225B4B30463946FAF75CFC28
:10AC300006460F4603229207554B28460399FAF71A
:10AC40000FFE07D20022534B28460399FAF74CFC1B
:10AC5000054603912068FAF771FD02460B4630461F
:10AC60003946FAF7B7FC07460A200791205EFAF743
:10AC700051FD3A46079BFAF745FC06460820099124
:10AC8000205EFAF735FD0021C943FAF77CFBFAF79D
:10AC9000D3FD3246099BFAF783FB06910890606862
:10ACA000FAF74CFD02460B4628460399FAF792FC48
:10ACB00005461A200E46205EFAF72CFD2A4633463A
:10ACC000FAF720FC0C9009911620205EFAF722FD7D
:10ACD000099B0C9AFAF764FB05910A902A463346C1
:10ACE00038460799FAF70EFC059B0A9AFAF70AFC10
:10ACF00005910A901420205EFAF70CFD3A46079B56
:10AD0000FAF700FC07461C200791205EFAF702FDC7
:10AD10002A463346FAF7F6FB0E900B911820205E78
:10AD2000FAF7F8FC0B9B0E9AFAF73AFB2A463346E1
:10AD3000FAF7E8FB0B910E902069FAF7EBFC0B9BFE
:10AD40000E9AFAF72DFB2A463346FAF7DBFB054647
:10AD50000E46E068FAF7DEFC2A463346FAF720FB97
:10AD60003A46079BFAF71CFB059B0A9AFAF718FB71
:10AD700001229207084BFAF7C5FB02460B46129CCC
:10AD80000898069903C411980CC0002026E700001B
:10AD9000FFFF5F4100007041E17A843F00B501216F
:10ADA000C9040300FFF755FC081A05080B0E11141F
:10ADB000171A0320C00400BD0720C00400BD0F20E7
:10ADC000C00400BD1F20400300BD3F20400300BD64
:10ADD0007F20400300BDFF20400300BD084600BDAA
:10ADE000FEB5264F0D4604000FD0002D0DD026468F
:10ADF00000202036B071F07129680D2088470028A6
:10AE000001DA7800FEBD102801D03846FEBDA562EB
:10AE1000E968002901D028208847204600F030F852
:10AE20000028F3DBA06AA52182680E209047A06A63
:10AE3000962182680F209047A06A022182686220D2
:10AE40009047A06A002182680E209047A06A0021E6
:10AE500082680F209047717930200191009006237D
:10AE6000202201212046FFF766FE0028CEDB204687
:10AE700000F0AEF80028C9DB0020FEBDFFFFFFFF99
:10AE800010B586B0044614216846FAF790F9002CF4
:10AE90007ED0A06A122143686A4610209847122883
:10AEA00077D1684600780122010168464078120394
:10AEB0000009081843492081884201DD801A208159
:10AEC0006846837840780007000D18186081884232
:10AED00001DD801A6081684600790122010168461F
:10AEE000C07812050003091868464079000908185F
:10AEF0003549E060884201DD801AE06068464079AB
:10AF00000007030B6846807900021B186846C07969
:10AF100018182061884201DD801A20616846417A54
:10AF2000007A0002081802B2284801210904A2820E
:10AF3000824201DD521AA2826A46D37A927A1202C2
:10AF40009A1812B2E282824201DD521AE2826A4605
:10AF5000537B127B12029A1812B22283824201DDC5
:10AF6000521A22836A46D37B927B12029A1812B23B
:10AF70006283824201DD521A62836A46537C127CEC
:10AF800012029A1812B2A283824204DD501A01E022
:10AF90000BE008E0A083A06A016828208847002809
:10AFA00006DA0120C04306B010BD0020C043FAE716
:10AFB000C011C0072034002800D08020607100201C
:10AFC000F1E70000FF070000FFFF0700FF7F000020
:10AFD00010B5040009D0A06A0721826808209047B4
:10AFE000002805DA0120C04310BD0020C04310BD79
:10AFF000072020342070002010BD0000FEB504465C
:10B000000020019000906079734940000E5A6178E9
:10B010002578491E7148CFB20163042D77D0072DE2
:10B0200075D000210291217801736C49E3790122E6
:10B0300092058969002B6CD0914381616748217A20
:10B040004173217A82698907890B0A438261002151
:10B05000042000F034FB324661492E2000F024FB2E
:10B060003846FFF7F3FB5F4E0522705D8100401804
:10B070005D49431807212B2000F030FB5B49029803
:10B0800001220B180B21282000F028FB705D584985
:10B0900080000A580C21282000F011FBE079554966
:10B0A00080004018A1794900425A0221272000F06F
:10B0B000FBFA51487E00825B0421272000F0F4FA5D
:10B0C000E079002829D0A07804282CD028206946CF
:10B0D000087220220621272000F0E6FA02AB0122A6
:10B0E0002621272000F0FAFA444938014018E17877
:10B0F000890042580821272000F0E1FAA17A601C5B
:10B10000627A0902114313D016E000E001E0012148
:10B1100088E71143F608816190E764220621272021
:10B1200000F0C2FAE0E71020694608720246D1E753
:10B1300033490172090A4172417A007A0A020243D4
:10B140002021272000F0B0FA2E4F0C2123203A684E
:10B1500000F0B5FAF01982880421232000F0A4FA47
:10B16000A07900280BD0E07927490122431800215B
:10B17000212000F0B3FA03200190012000902A075B
:10B18000120F10010243607800218007000B024378
:10B190000198000502430098400402432079C0064C
:10B1A000400902436079C00602431F2000F087FA7D
:10B1B000A07861780123084302040848DB03026198
:10B1C000E179490319430A4302610021082000F094
:10B1D00076FA0020FEBD00000CC6000880010020A9
:10B1E00004280000B4C5000824000020420000200C
:10B1F000BCC50008DCC50008E8C50008ECC50008AF
:10B2000041100000D4C500084400002038B50C46A9
:10B2100007498A8B002102432C2000F045FA68463A
:10B2200004706B46012206212C2000F057FA38BD2D
:10B230008001002010B5FFF7F5FA10BD10B50446E7
:10B240000421362000F0FCF80121C902002C01D0B5
:10B25000084300E0884302460421362000F02FFA1C
:10B2600010BD000038B540206946087000210E204E
:10B2700000F0E6F80446002211460E2000F01FFA06
:10B280006B46012200210D2000F028FA074A002118
:10B290000F2000F014FA00F0EDF9224600210E20F4
:10B2A00000F00DFA02480021017338BDF8FF272491
:10B2B000A0010020FEB50546042069460870514CE7
:10B2C0000020607521462031206348710873A083F7
:10B2D0006063A06300F0C8F84B4E206002E000F00D
:10B2E000C3F82060B042FAD10020FFF7CDFA00F099
:10B2F000BBF8464E20603078242801D9243806E077
:10B300000621F9F7F5FE0622101A4001084302064D
:10B3100001040A4301020A430243B2607060002143
:10B320001E2000F0CCF900F09FF820606B4601224F
:10B330000021242000F0D2F91E20FFF719FB86B26D
:10B34000300AA0730420FFF713FB074600F08CF8C7
:10B3500020603806000E0DD002206946087101AB4E
:10B36000012212212D2000F0B9F9A08B012109033F
:10B370000843A08300F078F820600620FFF7F8FA71
:10B3800060600720FFF7F4FAA060F006C00E207599
:10B3900001D110202075C0B200F0DCF9E80707D019
:10B3A000FFF7CDFAA08B0121C9020843A0830AE070
:10B3B0000521362000F02EF81549084002460521E7
:10B3C000362000F071F90120FFF75EFA0021042019
:10B3D00000F036F8A0610021262000F031F8152198
:10B3E0008903084302460021262000F068F9002264
:10B3F0002621362000F058F900F036F820600020B1
:10B40000FEBD0000800100203001CADE18000020CF
:10B41000FFFD000038B5094C89B280B26B460222AC
:10B4200000F028F8002806D16846407801026846F6
:10B430000078081884B2204638BD0000FFFF0000E5
:10B4400038B50024E44389B280B26B46042200F090
:10B4500011F8002806D103216846435C2202D41863
:10B46000491EFAD5204638BD10B500210846FFF721
:10B47000E7FF10BD38B5002909D0402420436C46B1
:10B480002070C8B27F2906D8607002200AE06946A1
:10B490000870012006E0802420436C466070C809D3
:10B4A000A0700320694600F0B7FF38BD10B5144600
:10B4B00003460A4621461120FFF7DCFF10BD10B5F8
:10B4C0000346052200211520FFF7D4FF10BD10B55B
:10B4D0000346052200211720FFF7CCFF10BD38B529
:10B4E000054600206946087000F0C4F8FF240134C6
:10B4F0002246002D01D00322120200210D2000F06F
:10B50000D3F8002D13D06B46012203210F20FFF743
:10B51000B1FF68460078000709D5FFF7A3FE224671
:10B5200000210D2000F0C0F80020C04338BD0020ED
:10B5300038BD10B5024601210A2000F0C0F810BD48
:10B5400010B5044600211A20FFF77AFF000D2203F0
:10B550000005120B024300211A2000F0B0F810BDC4
:10B5600010B5024602492E2000F09EF810BD0000E2
:10B5700004180000F8B505466B460122032104209B
:10B58000FFF778FF0126114C3607002D0DD02A4613
:10B5900000210C2000F088F8694608781021084343
:10B5A00069460870A069304307E069460878EF21D2
:10B5B000084069460870A069B0430B46A0610122AB
:10B5C0000321042000F08AF8F8BD0000800100206B
:10B5D00010B502460021182000F066F810BD0000EA
:10B5E000F8B50746002568460570B807204C2E467A
:10B5F00000280ADA8020694608706B460122002183
:10B600000D2000F06BF801202073F80769460878D8
:10B6100021D006210843694608706B4601220021AB
:10B620000D2000F05BF803210F20FFF7F3FE8121CE
:10B63000C900084219D04020694608706B460122B3
:10B6400000210D2000F04AF80020FFF7F7FD00254B
:10B650002673ED4309E002210843694608706B46F2
:10B66000012200210D2000F039F82846F8BD000025
:10B67000A00100201CB56B46012203210F20FFF71B
:10B68000F9FE684600784022C1091040C901400017
:10B69000814208D0012069460871024601AB0321AE
:10B6A0000D2000F01BF81CBD08B56B461A70120A7D
:10B6B0005A7089B280B2022200F010F808BD38B585
:10B6C00000236C46E254120A5B1C042BFADB89B29D
:10B6D00080B22346042200F001F838BD38B580243A
:10B6E000002909D0C02528436D462870C8B27F299B
:10B6F00007D86870022009E02043694608700120DD
:10B7000004E020436870C809A8700320694600F06F
:10B710002DFF38BD10B51446012312189B029A4222
:10B7200002D90020C04310BD0B46821E21460920CD
:10B73000FFF7D4FF002010BD10B5054A8905126936
:10B7400001430A4300210820FFF7B9FF002010BD84
:10B750008001002038B504466B4601220E212B20C3
:10B76000FFF788FE68460078E10640094001C90EEF
:10B770000143684601706B4601220E212B20FFF722
:10B78000ADFF38BD10B5002142541C06120A2243F9
:10B790001B0A491C0429F7DB10BD000013B5012367
:10B7A0001A4669460248FCF751FD00981CBD00008E
:10B7B000AC1500207CB5002425466846FFF77FFEC7
:10B7C00004206946220E2D02154322020C5C14430C
:10B7D000401EF7D5204629467CBD7CB50024254671
:10B7E0006846FFF774FE04206946220E2D021543B9
:10B7F00022020C5C1443401EF7D5204629467CBD2E
:10B80000FBF700FAFEF7FAF8FDF7F2F84149424873
:10B81000002522C005608561C56140490562C1609F
:10B820000838FBF78BFBFDF7CFF8FDF7E7F9FDF7DD
:10B8300083F9FDF795F8052601223607D103304636
:10B84000FBF7CBF9FDF758FEFCF77EFFFAF76EFA2F
:10B85000FAF73CFAFCF77CFD0721B015FFF7D6FCA0
:10B86000FFF7E8FC2E4C0A21208A0122484360841D
:10B8700011033046FBF7B1F92748C8222949C830DF
:10B88000FCF7B2FC284F294E207900283FD0607881
:10B8900000283CD0FEF7B2F82571FAF765FC20705D
:10B8A0000F280AD9012211033046FBF796F9FEF75B
:10B8B000F3F900220121090309E001225103304676
:10B8C000FBF78BF9FEF7E8F9002201214903304626
:10B8D000FBF783F9FCF764FE608C002801D0401E62
:10B8E00060841348618C00780843CDD138780028F3
:10B8F00001D00328C8D10121C9023046FBF760F905
:10B900000028C1D101210846FBF72CFCBCE7FCF75D
:10B9100047FEB9E7007C0040E4140020FFFF000070
:10B92000F4000020E40C00208100002000040050FE
:10B930005A00002010B586B01748FBF782FA142190
:10B940006846F9F734FC1548009003200190002068
:10B950000290052069460007FBF776F86946104813
:10B96000FBF772F869460F48FBF76EF801210846AD
:10B97000FBF7F8FBFF2401342046FBF7CBFB0A4919
:10B9800008680422104308602046FBF7D3FBFBF74E
:10B99000D9FB06B010BD0000E4140020FFFF00003A
:10B9A00000040050000800500070004010B5012253
:10B9B000920217491748FAF745FA154816490288BE
:10B9C0008A4223D00180FF2101318180FF21F5319E
:10B9D000C1800A21018100211E224181D24382813E
:10B9E0000122C28181831E23C38602230387782319
:10B9F00043878287C28702464032118451849184F2
:10BA0000C18391801421818200F02CFD10BD0000C3
:10BA1000AC0D002000FC0008AA550000F0B51FB4D2
:10BA200096B084460C460246199D1898039049002A
:10BA300068006300490840080193002A01D00126EC
:10BA400000E000269E19FE4BF6185B109E422BD399
:10BA50006E00039F0296002F00D00127F719F84EC1
:10BA6000F84BBE199E421FD3039E0346F64F334345
:10BA700009D03B469C4201D1002A04D0019B002AF8
:10BA800005D0012604E0002039461BB0F0BD002699
:10BA90009E19EE4B9E4207D8039F029E002F00D0B6
:10BAA0000127F6199E4207D92B4660462146189A6F
:10BAB000FEF782FE1BB0F0BD0023002C29DAE44E15
:10BAC000B04226DAE34EB04201DB022321E0DE4E33
:10BAD000B0421EDBE04E070DBE19142E09DD3427DF
:10BAE000BF1B039EFE400196BE40039FBE420BD08B
:10BAF0000FE0039F002F0CD11427BF1B0646FE400A
:10BB00000196BE40864204D1019BDE07F60F022358
:10BB10009B1B0E46164318D1002D16DA002C03D0BD
:10BB2000022B01D0012B06D00220FEF775FEFEF796
:10BB300039FE1BB0F0BD0220FEF76EFEFEF732FEAE
:10BB40000122D20751401BB0F0BD039E002E61D1EF
:10BB5000BF4EB04220D1C148844201D1002A08D052
:10BB6000B948814209DB002D10DB189829461BB02B
:10BB7000F0BD0020B4491BB0F0BD002D06DA012253
:10BB80002946D207189851401BB0F0BDB4497944FA
:10BB9000086849681BB0F0BDAB4FB84225D1002DF5
:10BBA0001FDA002904D0B14212D1002A09D018E0CE
:10BBB000002A72D1A649E20F0020D20711431BB020
:10BBC000F0BD0020E20F0146D20711431BB0F0BDCB
:10BBD000B14206DA234600203946F9F7FBFC1BB0D8
:10BBE000F0BD104621461BB0F0BDB14212DA01266D
:10BBF000B607B54203D1234610461946FEE3994ED7
:10BC0000B54207D1261E05DB1046314600F040FC48
:10BC10001BB0F0BD67007F081646002A40D10029FE
:10BC20000AD08B4A914229D1002C0EDD002D1CDB5D
:10BC3000002011461BB0F0BD022B16D0002C14D0F2
:10BC4000012B12D1002C14DB0FE0002C28DA002D80
:10BC500009DB012B03D000207D491BB0F0BD002083
:10BC600081491BB0F0BD012B03D0002001461BB061
:10BC7000F0BD00200121C9071BB0F0BD724A9142FE
:10BC80000ED1002C01DA002B17D0022B06D0002099
:10BC9000C043F9F73FFD1BB0F0BD90E20120F8E78B
:10BCA000E217521C94461A4307D000220892664CB1
:10BCB00062465B1E1A4307D009E00120FEF7ACFD87
:10BCC000FEF77EFD1BB0F0BD0022644C0892674A6F
:10BCD00090427DDD664B674A98421FDD914202DC4F
:10BCE000002D05DB4DE05848814217DB002D48DD73
:10BCF0000220FEF791FDFEF76BFD05460E46002281
:10BD0000534B21460898F9F7FDFB08467100490896
:10BD1000C00FC007014328461BB0F0BD914215DAA1
:10BD2000002D2EDA0220FEF777FDFEF751FD0546C5
:10BD30000E460022464B21460898F9F7E3FB7200B5
:10BD40005208C80FC0070243114617E03E4B994204
:10BD500023DD002D15DD0220FEF75EFDFEF738FD28
:10BD600005460E4600223A4B21460898F9F7CAFBD1
:10BD7000084671004908C00FC007014328461BB0A0
:10BD8000F0BD0220FEF748FDFEF72CFD49004908F2
:10BD9000E20FD20711431BB0F0BD002230463946F6
:10BDA000F9F7A2FB012205460E46D243F9F78AFCB9
:10BDB000314A324BF9F79EFB2A463346F9F7A2FB8C
:10BDC0000022284BF9F796FB07462A46334600E047
:10BDD00064E0039110461946F9F794FB3A46039B39
:10BDE000F9F790FB0746032209915207244B284696
:10BDF0003146F9F787FB07910C90224A204B3846D1
:10BE00000999F9F77FFB074601911F4A1F4B284606
:10BE10003146F9F777FB3A46019BF9F765FB074690
:10BE20000B460246099107990C98F9F7B9FA0025D3
:10BE30000E462846079B0C9AF9F756FB3A4627E030
:10BE4000FFFF1F00FFFF0F000000F03F0000E0FFBA
:10BE50000000F07F0000404301FCFFFF0000F0BF46
:10BE6000560B00000000E03F0000F0FF0000E04142
:10BE70000000F043FFFFEF3F555555555555D53F51
:10BE80004715F73FFE822B6544DF5DF80BAE543E4D
:10BE9000099BF9F72FFB02460B4652E101250020D2
:10BEA0002D05A94207DA352230463946F9F70AFC52
:10BEB00006463420C0430A151218FE481018039095
:10BEC0000803FD49000B01430F46FC49884201DC91
:10BED000002003E0FA49884202DA0120119005E0CF
:10BEE000002011900398401C7F1B03901198059728
:10BEF000C200F4480F9278448018436802683946BB
:10BF000030460D930292F9F7EFFA07910C90304604
:10BF10000D9B029A0599F9F743FA02460B46002059
:10BF2000E549F9F757FB09910490079B0C9AF9F73B
:10BF3000E9FA129000201090E3480D46784400681A
:10BF40000E90012178104907084311990D9B89042F
:10BF500040180121C90447183946029A0E98F9F78A
:10BF6000C3FA3246059BF9F7C5FA02460B46294645
:10BF70001098F9F7C7FA064602913B4629460E9AF1
:10BF80001098F9F7BFFA079B0C9AF9F7B3FA324603
:10BF9000029BF9F7A9FA099B049AF9F7B3FA0591FC
:10BFA000129A0A902B4610461946F9F7ABFA064644
:10BFB0000246C6480F460B4606217844FEF79CFB16
:10BFC00032463B460091049010461946F9F79AFA1A
:10BFD000009B049AF9F796FA06460F462B46194637
:10BFE000129A1098F9F7DCF9059B0A9AF9F78AFA80
:10BFF00032463B46F9F7D4F9109A079104902B4644
:10C0000010461946F9F77EFAB14E002233460991DF
:10C010000290F9F7C5F9079B049AF9F7C1F90020D6
:10C020000746024633460091F9F75EFA099B029AE9
:10C03000F9F75AFA079B049AF9F75CFA06460D914C
:10C040003A462946009B1098F9F75CFA07910C9044
:10C050002B463046129A0D99F9F754FA05460E46CA
:10C060003A46009B05990A98F9F74CFA33462A4656
:10C07000F9F796F902460B460746099107990C987D
:10C08000F9F78EF900250E462846079B0C9AF9F71A
:10C090002BFA3A46099BF9F72DFA07460722099130
:10C0A00052078C4B31462846F9F72CFA079100903D
:10C0B000894A884B38460999F9F724FA07460191CD
:10C0C000864A874B31462846F9F71CFA3A46019BC7
:10C0D000F9F766F9834B7B440F9A9B181A685B68E3
:10C0E000F9F75EF9029009910398F9F713FB0591AE
:10C0F0000490099B029A07990098F9F751F97A4B35
:10C100007B440F9A9B181A685B6817460393F9F7EC
:10C1100047F9059B049AF9F743F90E462846059B13
:10C12000049AF9F7E1F93A46039BF9F7DDF9079B21
:10C13000009AF9F7D9F9099B029AF9F7DBF9024657
:10C140000B46199900200C900F461898F9F7DAF968
:10C15000029104903B460C9A19991898F9F7C4F982
:10C160002A463346F9F7CEF9029B049AF9F718F9F3
:10C1700009910E902A46334639460C98F9F7C2F9D0
:10C1800006460F46099B0E9AF9F70AF9574A0D46DB
:10C19000914220DB5242AA18024310D132463B465C
:10C1A000F9F7A2F904900391514A524B09990E985C
:10C1B000F9F7F6F8039B049AF9F752FB1ED2022016
:10C1C000FEF72AFBFEF704FB49004908E20FD207FD
:10C1D00011431BB0F0BD6A00474B52089A420DD381
:10C1E000464AAA18024300D0CBE532463B46F9F74F
:10C1F0007BF9099B0E9AF9F733FBF5D96800002308
:10C2000040082C490393020D3D4B5218984223DD00
:10C2100001200005521CD04042195000400D40182A
:10C2200038497944096813468C463749C1408B43E5
:10C2300012030121120B090551181422101AC140D2
:10C240000391002D01DA4842039062463046394698
:10C25000F9F74AF906460F4632463B4609990E98C9
:10C26000F9F79EF800252A46284B28460591F9F74C
:10C2700049F907910C90264A264B28460599F9F76B
:10C2800041F90091029032463B4628460599F9F75C
:10C290002BF9099B0E9AF9F72DF91F4A1F4BF9F755
:10C2A00031F9009B029AF9F77BF807460B460246E4
:10C2B000099135E001FCFFFF0000F03F8E9803007C
:10C2C0007AB60B0066070000A8070000D20600003F
:10C2D0000000084009C7EE3FFD033ADCF5015B149E
:10C2E000E02F3EBEA60500006C0500000000904057
:10C2F000FE822B654715973C00CC904000346F3F81
:10C300000000E03FC2040000FFFF0F00432EE63FA5
:10C31000396CA80C615C20BEEF39FAFE422EE63F74
:10C3200007990C98F9F73CF805460E46079B0C9ABE
:10C33000F9F7DAF83A46099BF9F7DCF809912A4649
:10C3400033460E9010461946F9F7DCF807460246C8
:10C350002F480B46059105217844FEF7CDF93A4662
:10C36000059BF9F7CFF82A463346F9F7C3F8074695
:10C37000019128463146099B0E9AF9F7C3F8099BAB
:10C380000E9AF9F70DF8012304910C9000229B07F7
:10C3900038460199F9F7A8F805910E903A462846D3
:10C3A0003146019BF9F7AEF8059B0E9AF9F712F9A1
:10C3B000049B0C9AF9F798F82A463346F9F794F853
:10C3C0000022144BF9F796F8064603980D4600052F
:10C3D00041190915002912DC30462946039AF9F75C
:10C3E00071F9FEF743F9042801D1FEF7FBF9304655
:10C3F0002946039AF9F766F9064601E004E0291890
:10C400000B46324621460898F9F77CF81BB0F0BD80
:10C41000640300000000F03FF0B58C4600251026B4
:10C42000052109078E620E4C08E067467F5DE760D4
:10C43000A768FF07FCD0E7681F706D1C8542F4DB1E
:10C440000020074606E0E760A568ED07FCD0E56838
:10C450001D54401C9042F6D38E610020F0BD0000B8
:10C460000030014070B572B60124074DA402214688
:10C470002846F9F7CDFC002804D022460349284677
:10C48000F9F76AFD62B670BD00FC0008AC0D002033
:10C49000F8B506460C46F9F7F1FA051E0F4600D02E
:10C4A0000120014349000B484908411AC90F0DD02A
:10C4B000002E01D0012100E000210C436100490859
:10C4C000401AC00F02D10120FEF7A6F928463946CE
:10C4D000F8BD00000000F07FF8B515460E4607468F
:10C4E000002407E03819C0B200F008F8641C287076
:10C4F000E4B26D1CB442F5D33046F8BD10B5044625
:10C50000FBF7EAFFEE20FBF7BAFFFCF71EF8204628
:10C51000FBF7B5FFFCF719F8FBF7DEFFEF20FBF7A1
:10C52000AEFFFCF712F80020FBF77CFF0446FBF798
:10C53000EEFF204610BD704770B50D460446FBF770
:10C54000CBFFEE20FBF79BFFFBF7FFFF2046FBF73F
:10C5500096FFFBF7FAFF2846FBF791FFFBF7F5FF85
:10C56000FBF7D5FF0A20FEF7A0FA70BDF0B5002555
:10C57000102605279C463F070B46BE620C4C06E082
:10C58000595DE160A168C907FCD0E1686D1C854276
:10C59000F6DB002007E06146095CE160A168C9079D
:10C5A000FCD0E168401C9042F5D3BE610020F0BD94
:10C5B000003001400000010203040005405C00005F
:10C5C000A05C0400C06C0800805C0400E03F1E001A
:10C5D000E07D1E0007A9022570889B880A001600CE
:10C5E000010006000100020087008D002D001A31B5
:10C5F00052001A339A001A351D011A376B003B316D
:10C60000BE003B335E013B3596023B370000995933
:10C610009959EB518F421E45142E0080EB51F5289D
:10C620003333E13A703DE13AC235852BC2353333BD
:10C63000C235C235AE47E13A5138A3305138000017
:10C6400000000000000001020304060708090304BB
:10C6500006080C101820300000000001020304003E
:10C66000000000000000F03F000000000000F83F64
:10C6700000000000000000000000004003B8E23F9E
:10C68000000000000000000006D0CF43EBFD4C3E50
:10C69000033333333333E33FFFAB6FDBB66DDB3F45
:10C6A0004D268F515555D53F01411DA96074D13F8D
:10C6B00065DBC9934A86CD3FEF4E454A287ECA3F87
:10C6C0003E5555555555C53F93BDBE166CC166BF09
:10C6D0002CDE25AF6A56113FF16BD2C541BDBBBE02
:10C6E000D0A4BE726937663E000000000000000062
:10C6F00010C700080000002054010000445B00083F
:10C7000050C70008540100208419000008A8000840
:10C710000124130704380D091E08054008260910D6
:10C720004008560A131D043B08BE0516D8BC40102D
:10C730000852010334C842035A5C121B0202BD14A2
:10C74000090102628149A80146294C920492200005
:04000005080050C1DE
:00000001FF
